:10800000004000208519010095EB000095EB000071
:1080100095EB000095EB000095EB000000000000E0
:1080200000000000000000000000000095EB0000D0
:1080300095EB00000000000095EB0000FD850000BE
:1080400095EB000095EB000095EB000095EB000030
:1080500095EB000095EB000095EB000095EB000020
:1080600095EB000095EB000095EB000095EB000010
:1080700095EB000095EB000095EB000095EB000000
:1080800095EB000095EB000095EB000095EB0000F0
:1080900095EB000095EB000095EB000095EB0000E0
:1080A00095EB000095EB000095EB000095EB0000D0
:1080B00095EB000095EB000095EB000095EB0000C0
:1080C00095EB000095EB000095EB000095EB0000B0
:1080D00095EB000095EB000095EB000095EB0000A0
:1080E00095EB000095EB000095EB000095EB000090
:1080F00095EB00000D88000095EB000095EB00006B
:1081000095EB000095EB000095EB000095EB00006F
:1081100095EB000095EB000095EB000095EB00005F
:1081200095EB000095EB000051E6000095EB000098
:1081300095EB000095EB000095EB000095EB00003F
:1081400095EB000095EB000095EB000095EB00002F
:1081500095EB000095EB000095EB000095EB00001F
:1081600095EB0000A5FD000095EB000095EB0000ED
:1081700095EB000095EB000095EB000095EB0000FF
:1081800095EB000095EB000095EB000095EB0000EF
:1081900095EB000095EB000095EB00004DEA000028
:1081A00095EB000095EB000095EB000095EB0000CF
:0C81B00095EB000095EB000095EB000043
:10840000FFFFFFFFFFFFFFFFFFFFFFFF7EF9FFFF03
:1084100010B5054C237833B9044B13B10448AFF3BE
:1084200000800123237010BD00C6FF1F0000000064
:10843000E01D01000C4B43B10C480D4910B5AFF3E2
:1084400000800C48036823B910BD0A48036833B99B
:108450007047094B002BF7D0BDE810401847064B7A
:10846000002BF5D0184700BF00000000E01D010000
:1084700004C6FF1F6CC5FF1F0000000080F31188B9
:1084800070472F4B41F238015A5842F478525A50F3
:108490002C4A927902F00C020C2A4FD041F244028D
:1084A0002949995003F558339A78110748BF9A78AB
:1084B000264944BF42F008029A70214B41F244021F
:1084C000995041F204015A5842F4803242F0C002FD
:1084D0005A501A6842F440221A6003F5E833242205
:1084E0005A701B4A80211170A2221A70DA7802F0A9
:1084F0001F02DA7007221A710C225A719A799207B8
:10850000FCD59A79D006FCD40E4B19469A7902F024
:108510000C02082AFAD14C225A718B7903F00C0311
:10852000082BFAD1074B1A4699794906FCD5222126
:108530001970937903F00C030C2BFAD1704700BF2C
:1085400000700440004006400000330100001301A9
:1085500000500640264B5A7902F0E0025A711A790F
:1085600002F0F8021A71A3F500531A7802F08C0297
:1085700042F050021A705A7802F09C0242F0400217
:108580005A709A7802F0E6029A701A4A0023137021
:1085900083F31188184B012283F8182383F81923D9
:1085A000022283F8582383F8592383F81D2383F884
:1085B0001E2383F81F2383F8202383F8212303221B
:1085C00083F82D2383F82F2383F8312383F8332373
:1085D00083F83523042283F83923052283F83A23CC
:1085E000062283F85723072283F84923704700BFE8
:1085F00000F0074000E0074000E100E0314A136866
:108600000133F0B51360304A1368013313602F4B08
:108610001A683AB11A68013A1A601B6813B92C4BF0
:1086200001221A702B4B1A6812B11A68013A1A60AB
:10863000294B5A68294B92B21A60294A1868116866
:10864000884223DD19681068264C091AB1F5004FDD
:1086500025480ADA1E6817682168D0E90045F61B2C
:108660007143641845EBE1750BE0196817682668DB
:10867000D0E90045C91BC1F580317143641A65EB2F
:10868000E175C0E900451B681360F0BD186811680A
:108690008842F8DA11681868124C091AB1F5004FCF
:1086A000114806DA16681F682168F61BD0E90045F4
:1086B000E3E711681F682668C91BD0E90045C1F5CA
:1086C0008031CDE71CC6FF1FFCCFFF1F10CDFF1F61
:1086D0000CCDFF1F14CDFF1F009003402CCDFF1FBA
:1086E00020CEFF1F64CDFF1F68CDFF1F41F23C026B
:1086F00005498B5843F000738B50044B044A5A6071
:1087000007221A60704700BF0070044010E000E0CC
:1087100040190100014B1868704700BF1CC6FF1FBD
:108720001449154B41F23402072888BF002010B5C8
:1087300053F82030114CB4FBF3F48B5843F48063AE
:108740008B500F4B4FF400725A602D209A6006F048
:1087500039FA0C4B0022DA709A709A71DA725A71F7
:10876000C4F30422E4B21A705C70DA7842F02C028E
:10877000DA7010BD00700440201C010020AA4400E3
:108780000090044000A00640094A13685168013374
:10879000202B08BF00238B4208D0116811440872B7
:1087A0001360044AD37843F08003D370704700BF4E
:1087B00020C6FF1F00A006400A4B996ADA6A914260
:1087C0000DD09A6A511C1A44996292F830200270B6
:1087D0009A6A202A01D100229A6201207047002063
:1087E000704700BF20C6FF1F044B1A7802F0FF003D
:1087F00012B100221A700120704700BF0CCDFF1F7C
:10880000014B1865704700BF20C6FF1F30B52648D2
:108810000179C9B28C0617D5244BDA6A9C6A0132F9
:10882000202A08BF0022A2421BBFDC6AC579C27998
:1088300018191EBFEDB280F83050DA621C4A0520CC
:1088400010601A6D1B4B1A604A0608D51A4B4FF47C
:1088500000329A60144AD37803F0BF03D3700B063A
:108860001BD5144B1868C0B9104B19685A6891424F
:1088700014D0114A4FF4003151605A68511C1A4407
:108880005960117A084AC9B2D1715968202908BFC4
:108890005860D37843F04003D37030BD024AD37898
:1088A00003F07F03F8E700BF00A0064020C6FF1FCB
:1088B00010CDFF1F14CDFF1F00F00F4062B67047B0
:1088C000FFF7FCBF72B67047FFF7FCBF4FF0E02325
:1088D00018B1034AC3F80C2D7047024AFAE700BFEB
:1088E0000400FA050100FA0510B9C90801F0D8BC66
:1088F0007047F7B5454A464E46494FF480731361B9
:1089000053619363D363136453647161B1604249EB
:1089100040F20310086048608860C8608862C862DE
:108920000B644B6401F5352140314FF44030486110
:1089300048603A493A480B6040F607044B608B6048
:10894000CB62446144603748036043608360C36026
:10895000036100F53320C0301424446104244460D2
:1089600010248460304C636104F5322404F5807473
:108970002025656141F204042C4D2F5927F0E007B2
:108980002F512F5947F0C0072F514FF4A064CC60EE
:1089900013603446D360082600230A211A46B446E1
:1089A0001F46A646C4F804C00197019DB5F57A7F1D
:1089B00021D3DEF81050A660ED0748BF01320197C1
:1089C000019DB5F57A7F1AD3DEF81050ED0758BF38
:1089D00001330139E6D10A2A154A14D10A2B12D1E2
:1089E00001231370094B4FF4E0621A60DA60102320
:1089F000436003B0F0BD019D01350195D5E7019DB0
:108A000001350195DCE70023EBE700BF009004404F
:108A100000F00F402880030000A0044000B0044094
:108A200080F00F4000C0044000D0044000700440BB
:108A300060CDFF1FF7B5114B1B78E3B1104911480A
:108A4000114D20231E4600240F4686464E60866048
:108A50000194019AAA420AD9BB60CEF8043001946D
:108A6000019AAA42F2D8019A01320192F8E7019ADA
:108A700001320192EDE703B0F0BD00BF60CDFF1FF2
:108A800000F00F4000F10F401FA10700072809D890
:108A9000DFE800F004090C0F111416184FF400421F
:108AA0000A4B5A6070474FF48032F9E70222084BB4
:108AB000F7E70822FBE74FF40062F8E70122F6E748
:108AC0000422F4E74FF48062F1E700BF00F00F40AA
:108AD00040F00F40072809D8DFE800F004090C0F28
:108AE000111416184FF400420A4B9A6070474FF465
:108AF0008032F9E70222084BF7E70822FBE74FF440
:108B00000062F8E70122F6E70422F4E74FF48062FE
:108B1000F1E700BF00F00F4040F00F4010B500211A
:108B2000044644FA01F3DB07C8B205D5FFF7AEFFF0
:108B300001310829F5D110BDFFF7CCFFF8E708B5E2
:108B400006282CD8DFE800F0040D12171C2126009F
:108B5000002005F0C1FDB0F5806F34BF002001207A
:108B600008BD104B186900F0010008BD0D4B1869D5
:108B7000C0F3800008BD0B4B1869C0F3802008BD0E
:108B8000084B1869C0F3400008BD064B1869C0F3D4
:108B9000C00008BD034B1869C0F3C02008BD002009
:108BA00008BD00BF40F00F4007282DD8DFE800F0D7
:108BB00004090E13181D2227144B1868C0F3C03087
:108BC0007047124B1868C0F300407047104B18688C
:108BD000C0F3400070470E4B1868C0F3C0007047E8
:108BE0000B4B1868C0F3C0207047094B186800F0A1
:108BF00001007047064B1868C0F380007047044BB3
:108C00001868C0F3802070470020704700F00F40C4
:108C100040F00F4070B5002425460126E0B2FFF772
:108C20008EFF18B106FA04F31D43EDB20134082C8F
:108C3000F4D1284670BD10F0010F314B33D05A6982
:108C400042F002025A614FF400329A6010F0020FB3
:108C50002C4A30D0596941F00801596102219160D4
:108C600041072FD5596941F4006159614FF4006102
:108C7000916001072ED5596941F0010159614FF406
:108C800080319960C1062DD5596941F004015961BF
:108C90000121916081062CD5596941F480615961A7
:108CA0000423936070474FF400325A605A6922F0EF
:108CB00002025A61CAE702215160596921F0080194
:108CC0005961CDE74FF400615160596921F40061A9
:108CD0005961CEE74FF480315960596921F00101A3
:108CE0005961CFE701215160596921F004015961AF
:108CF000D0E7042151605A6922F480625A617047BA
:108D000040F00F4080F00F401B4B5A6810F0010FED
:108D100014BF42F0030202F002025A60DA688107CF
:108D20004CBF42F0030202F00202DA60124BDA6A30
:108D300010F0040F14BF42F0030202F00202DA62E4
:108D40001A6801074CBF42F0030202F002021A60E7
:108D5000094B9A6810F0100F14BF42F0030202F0A2
:108D600002029A609A6A81064CBF42F0030202F046
:108D700002029A62704700BF00A0044020B9034B72
:108D80001869C0F3403070470020704700F00F4072
:108D900008B5082005F0A0FC5E280DD90F4B1A7805
:108DA0000AB901221A70082005F096FC63280BD935
:108DB0000B4B04229A6008BD082005F08DFC542856
:108DC000F1D80022054BEDE7082005F085FC54287A
:108DD0009EBF034B04225A6008BD00BF74C6FF1F2C
:108DE000C0F00F40034B1878013801288CBF0020D9
:108DF0000120704774C6FF1F034B1878012806BF77
:108E000002221A700020704774C6FF1FC0B201F022
:108E100071BBC0B201F064BB08B507F0E7FD06F016
:108E2000A5F806F055F8BDE8084007F061BE38B572
:108E3000054605F0A3FF08280AD9002428190134A3
:108E400006F01CF8092CF9D106F04CF8012038BDC9
:108E5000002038BD092105F0B1BF002006F03EBA60
:108E60002149224841F23C028B5843F440538B5035
:108E70001F4B012119601A6802431A601D4ADA600B
:108E80001A61DA6A42F08052DA621A6822F001024C
:108E90001A601A6822F000621A6003F5F8334FF482
:108EA00000721A615A619A61DA61A3F5F0331960B0
:108EB0001968014319601049D96001F52001196151
:108EC000D96A41F08051D962196821F00101196015
:108ED000196821F00061196003F500331A605A60C7
:108EE0009A60DA601A61704700700440000C1F80BD
:108EF00000C002400300013E0400513EFF281ED87E
:108F000000041E4B00F47C108AB141F0006108435C
:108F10005863DA6A002AFCDA184BDA6AD100FCD509
:108F2000986BDA6A42F01042C0B2DA62704741F0E0
:108F3000004108435863DA6A002AFCDAF0E7B0F52A
:108F4000007F18D200040E4B00F47C105AB141F09F
:108F5000006108435863DA6A002AFCDA084BDA6ACF
:108F6000D200FCD5DCE741F0004108435863DA6ADF
:108F7000002AFCDAD4E70020704700BF00C002409E
:108F800000D00240C0EBC00038B500220C4600F50E
:108F9000006503210120FFF7B1FF0022C5F307217F
:108FA0000120FFF7ABFF0022E9B20120FFF7A6FF87
:108FB000002211460120FFF7A1FF00221146207078
:108FC0000120FFF79BFF0022114660700120FFF790
:108FD00095FF00221146A0700120FFF78FFF0022AD
:108FE0001146E0700120FFF789FF00221146207131
:108FF0000120FFF783FF0122607100211046FFF777
:109000007DFFA07138BD38B54FF400640122062100
:109010001046FFF773FF002205210120FFF76EFFC6
:10902000012200211046FFF769FF8007F3D50022D7
:1090300002210120FFF762FF0022C4F30721012073
:10904000FFF75CFF0022E1B20120FFF757FF002588
:10905000A5F13F014A424A41012000210135FFF7B5
:109060004DFF402DF4D1002205210120FFF746FFDE
:10907000012200211046FFF741FFC307F3D440341B
:10908000B4F5804FC2D138BDF7B5C0EBC00000F5D4
:1090900000650C46002203210120FFF72FFFC5F3D6
:1090A000072100220120FFF729FFE9B20022012059
:1090B000FFF724FF002211460120FFF71FFF0022C7
:1090C000114607460120FFF719FF00221146064608
:1090D0000120FFF713FF0022114605460120FFF78C
:1090E0000DFF002211468DF803000120FFF706FF57
:1090F000002211468DF804000120FFF7FFFE012237
:109100008DF8050000211046FFF7F8FE23788DF852
:109110000600BB420ED16378B3420BD1A378AB42B9
:1091200008D1DDF80300D4F80330C31A584258417F
:1091300003B0F0BD0020FBE7012238B504460D4620
:1091400010460621FFF7DAFE002205210120FFF775
:10915000D5FE012210460021FFF7D0FE8207F3D58D
:10916000002202210120FFF7C9FE0022C4F30721DB
:109170000120FFF7C3FE0022E1B20120FFF7BEFE8F
:10918000012229461046FFF7B9FE002205210120E1
:10919000FFF7B4FE012200211046FFF7AFFEC30720
:1091A000F3D438BD38B50D46C0EBC00404F50060FB
:1091B0000978FFF7C1FF697804F60100FFF7BCFFEB
:1091C000A97804F60200FFF7B7FFE97804F6030078
:1091D000FFF7B2FF297904F60400FFF7ADFF6979C4
:1091E00004F60500FFF7A8FFA97904F60600BDE81C
:1091F0003840FFF7A1BF2DE9F84316460122044687
:10920000884610460621FFF779FE0022052101203D
:10921000FFF774FE012200211046FFF76FFE85075D
:10922000F3D5002202210120FFF768FE0022C4F3DB
:1092300007210120FFF762FE0022E1B20120FFF7C3
:109240005DFE0025771EB5420DD1002205210120CB
:10925000FFF754FE012200211046FFF74FFEC3071F
:10926000F3D4BDE8F883013414F03F0918F8051071
:1092700039D0781B424242410120FFF73FFEB9F14D
:10928000000F2ED1BD422CD2002205210120FFF774
:1092900035FE012200211046FFF730FEC107F3D44E
:1092A000012206211046FFF729FE00220521012098
:1092B000FFF724FE012210460021FFF71FFE820760
:1092C000F3D5002202210120FFF718FE0022C4F38B
:1092D00007210120FFF712FE0022E1B20120FFF773
:1092E0000DFE0135AFE70122C6E710B500220446A6
:1092F00003210120FFF702FEC4F307210022012011
:10930000FFF7FCFDE1B200220120FFF7F7FD01228B
:1093100000211046BDE81040FFF7F0BDF8B5044647
:109320000E461546032100220120FFF7E7FDC4F396
:10933000072100220120FFF7E1FDE1B20022012018
:10934000FFF7DCFD77193446013DBC4200D1F8BD82
:10935000A21BAB1A5A425A4100210120FFF7CEFD51
:1093600004F8010BF1E7F7B5002205210120FFF712
:10937000C5FD012200211046FFF7C0FD10F0710469
:10938000F2D1FFF7C7F90546FFF7C4F9401B0028E3
:10939000B8BF4042B0F5FA6F22DAC4B1334B1B7844
:1093A00003BB402232490020FFF7B8FF2022314999
:1093B0004020FFF7B3FF20222F496020FFF7AEFFC8
:1093C00020222E498020FFF7A9FF03B0F0BD40F214
:1093D000FF70FFF78AFFA0F1AA035C425C41D3E76C
:1093E000002CDBD1002140F2FF70FFF7A5FEFFF754
:1093F0000AFE40221E49224F224E0020FFF7FBFEAC
:1094000040254FF480742046B4223946FFF7F3FE1E
:10941000B434284620223146FFF7EDFEB4F5477FED
:1094200005F12005EFD102AD002345F8043D4FF4CE
:10943000C3642046042229460434FFF7DCFEB4F559
:10944000FF6FF6D1002301934FF4A7642046042256
:1094500029460434FFF7CFFEB4F5C36FF6D1AA2135
:1094600040F2FF70FFF768FE9BE700BF60CDFF1F73
:109470000CC0FF1FC0CDFF1FE0CDFF1F00CEFF1FA0
:10948000701C0100501C01002DE9F0411378C3F35A
:10949000411507460E46144615BB3D4A117BF9B9E6
:1094A000D8071DD45F2B1BD83A490978C1B913F0EE
:1094B000970F15D1DFF8E48098F800302BB1517A7E
:1094C0002846FFF711FA88F80050DFF8D48098F8A2
:1094D00000302BB1002001F00DF8002388F8003097
:1094E0000022217840F20110FFF708FD30700022C1
:1094F000617840F20110FFF701FD70700022A17841
:1095000040F20110FFF7FAFCB070E178012240F25E
:109510000110FFF7F3FCF0702378D90735D45F2BE7
:1095200033D803F01E03082B11D0142B24D0062BA4
:109530002BD124237B430C2707FB0537164DA2783C
:10954000E3783D4443EA02236B60BDE8F081A278F2
:10955000E378114943EA0223242257430C2202FBF9
:1095600005754B51A27812070FD56FEA03536FEAC6
:1095700013534B51BDE8F08124235F430C2303FBBD
:109580000575054BE2781D442A72BDE8F08100BFE5
:10959000C0CDFF1F7CCEFF1F70CDFF1F79CEFF1FF8
:1095A0007FCEFF1F07B513788DF8013053788DF803
:1095B00000108DF8023001A993788DF803306A46C7
:1095C000FFF762FF03B05DF804FB07B58DF80010EC
:1095D0008DF801208DF802306A469DF810308DF824
:1095E000033001A9FFF750FF03B05DF804FB07B596
:1095F00000238DF800108DF801308DF80320131230
:1096000001A96A468DF80230FFF73EFF03B05DF80E
:1096100004FB5F292DE9F34180460F46144606D826
:1096200017F01E064FEA511113D0022E2ED023142C
:109630008DF801306A46231201A940468DF800706A
:109640008DF802308DF80340FFF71EFF02B0BDE831
:10965000F081032212FB0012244B2548120103EB78
:10966000020E9C50DEF80410651A002DB8BF6D4242
:10967000854208DD13448C424FF00102CCBF0C1828
:109680000C1A1A73D3E78EF80C60D0E7032616FB8A
:109690000016164D3601AA1955F806E05460AEEBD7
:1096A000040024F07F4300289360114BB8BF404270
:1096B000984217DD7445B4BF1B19E31A4A018DF8AF
:1096C00000201A148DF801201A128DF8022001A929
:1096D0006A46404635448DF80330FFF7D5FE012336
:1096E0002B73A4E700231373A1E700BFB4CEFF1FC1
:1096F000FFFF7F0007B511F01C0204D1FFF789FFBF
:1097000003B05DF804FB00238DF800106A4601A940
:109710008DF801308DF802308DF80330FFF7B4FE7C
:10972000EEE70122114640F20110FFF7E7BB13B547
:10973000144602AA41F0010102F8041D6946FFF730
:10974000A3FE9DF8013023709DF8023063709DF8F0
:1097500000009DF80330A37002B010BD07B502AA47
:1097600041F0010102F8041D6946FFF78DFEBDF8C6
:10977000020040BA80B2030544BF6FEA00506FEAAE
:10978000105003B05DF804FBF7B5490102AD4CB2CF
:1097900044F0150305F8083D174601A92A46064678
:1097A000FFF772FE9DF805308DF8013044F0140487
:1097B0009DF806308DF800402A4601A930468DF804
:1097C00002308DF80370FFF75FFE03B0F0BDF7B510
:1097D000490102AD4CB244F0150305F8083D1746A7
:1097E00001A92A460646FFF74FFE9DF805308DF881
:1097F000013044F014049DF807308DF800402A46EB
:1098000001A930468DF802708DF80330FFF73CFE59
:1098100003B0F0BD73B502AC7F2304F8083D0D46DC
:10982000224601A90646FFF72FFE7E238DF8003061
:109830009DF805308DF8013005F00F059DF80730D3
:109840008DF80250224601A930468DF80330FFF70B
:109850001BFE02B070BD2DE9F74F400145B2C1F3C8
:109860000A0845F0180101AA01F0F8010020FFF7ED
:109870005EFF9DF805404FEA141904F00F04A1455E
:1098800040465CDC07F08AFAA4EB09040646012096
:10989000A0400F4607F092FA0022334B07F0F4FA8B
:1098A00002460B463046394607F018FC07F026FD05
:1098B00007F096FA2AA3D3E9002307F0E5FA07F0A8
:1098C0001DFD07F08DFA0022284B07F0DDFA4FF05E
:1098D000FF3906460F46CA4600244FF0010B0BFA2B
:1098E00004F007F06BFA3B46324607F0CDFA07F07A
:1098F000DDFCA0F180037F2B98BFA14604F1010499
:1099000098BF82460E2CEAD1002445F0120101AA2C
:10991000204601F0F2018DF804408DF805A08DF885
:109920000690FFF73FFE45F00C012046424601F04D
:10993000EC01FFF75CFE204603B0BDE8F08F07F0B6
:109940002DFAA9EB040406460120A0400F4607F0BB
:1099500035FA02460B460020034907F0BFFB9FE79C
:1099600004560E2DB29DEF3F0000604000002040E5
:1099700073B54A0803244FF4807314FB0233B424F4
:1099800014FB0034064620460D46FFF7AEFC8DF86A
:109990000400601CFFF7A9FC8DF80500A01CFFF770
:1099A000A4FC45EA46118DF8060001AAC9B20020C0
:1099B000FFF7F8FD02B070BD73B50D4641EA4011E6
:1099C00001AA0646C9B20020FFF7B1FE03244FF4F6
:1099D00080736D0814FB0535B42414FB06549DF800
:1099E00004102046FFF7A8FB9DF80510601CFFF748
:1099F000A3FB9DF80610A01CFFF79EFB02B070BDF4
:109A000010B5C4B221466401E4B202220020FFF77F
:109A1000BBFE44F008010020FFF76CFE44F00A0191
:109A20000020BDE81040FFF765BE37B5440144F0A3
:109A30001604E4B20D4601AA21460020FFF777FE86
:109A40009DF8053015F0010F14BF43F0400323F0DB
:109A500040038DF805309DF8053015F0020F14BF56
:109A600043F0100323F01003002001AA21468DF8D3
:109A700005308DF80600FFF795FD03B030BD37B512
:109A8000440144F01604E4B20D4601AA2146002028
:109A9000FFF74DFE9DF8053015F0010F14BF63F080
:109AA0007F0303F07F038DF805309DF8053015F036
:109AB000020F14BF43F0200323F02003002001AA6B
:109AC00021468DF805308DF80600FFF76BFD03B0D9
:109AD00030BD07B5410141F0160101AA01F0F601C0
:109AE0000020FFF724FE9DF80530C3F38010DB064D
:109AF00048BF40F0020003B05DF804FB07B5410128
:109B000041F0160101AA01F0F6010020FFF70FFE57
:109B10009DF80530D8099B0648BF40F0020003B00D
:109B20005DF804FB70B5104C05016219204693687E
:109B30008B420DDACB1AC3F18076B342546804DC51
:109B4000234453602844816070BDA41B5460F9E72E
:109B5000F8DD5B1AC3F18076B342546801DCE31A86
:109B6000EFE73444F2E700BFB4CEFF1F73B502AA9B
:109B700041F001030C4602F8043D69460546FFF733
:109B800083FC9DF802009DF80110000240EA0140AC
:109B90009DF803100843030248BF40F07F405F2C4C
:109BA00005D8660914F01E0403D0022C08D002B0B8
:109BB00070BD032010FB05600001094B1858F6E743
:109BC00005EB4503334420F07F41D8B2FFF7AAFFED
:109BD000032010FB0560024D05EB00156868E6E701
:109BE000B4CEFF1F38B50D4668210446FFF7BEFF0F
:109BF0003DB140F0010220466821BDE83840FFF742
:109C000008BD20F00102F6E773B51C4B587E10F03A
:109C100001001DBF40F22312682100204FF4917211
:109C200008BF6821FFF7F5FC0223009300231A46C2
:109C30007E211846FFF7C9FC00240025E6B2E9B2F0
:109C400030460135FFF794FE1D2DF8D17501EDB2B8
:109C500045F00C010020FFF789FF01463046FFF771
:109C6000FAFD013443F2FF1245F016010020FFF720
:109C7000BEFC032CE1D102B070BD00BF0CC0FF1FC1
:109C80007FB5450104AA45F0030302F8043D0446EC
:109C900002A90020FFF7F8FB9DF80A309DF8091093
:109CA0001B0243EA01439DF80B1020461943FFF7BE
:109CB00039FF134A2301D118087BE8B111480C265B
:109CC00006FB0404267ABEB9D2584B680E48D41A53
:109CD000002CB8BF6442844210DD9A42CCBF1A18EF
:109CE0001A1AD3B2009305F0E001C2F30723002053
:109CF000C2F30742FFF769FC04B070BD0E73F0E7D2
:109D0000B4CEFF1F70CDFF1FFFFF7F0038B5C0F33B
:109D10000741054600224FF48170FFF7EFF80C4C25
:109D2000000220600022C5F307214FF48170FFF785
:109D3000E5F823681843000220600122E9B24FF4DD
:109D40008170FFF7DBF8236818430009206038BDF5
:109D500078C6FF1F10B5244CC00023181A79032AB7
:109D600084BF03221A7123189A79032A84BF03221D
:109D70009A7123181A7A0F2A84BF0F221A72231895
:109D80005A7A072A84BF07225A7223189A7A0F2A0E
:109D900084BF0F229A72221813795279DB0343F49D
:109DA0000021E16012B143F40423E3602318DB795E
:109DB0001BB1E36843F40053E3602044037A8279E3
:109DC000DB0143EAC223E2681343427A43EA021307
:109DD000C27AE36012B9827A1343E360E068FFF766
:109DE00095FFE368236110BD78C6FF1F10B5104CC6
:109DF0000023C000E36023185B7E13B14FF40073AF
:109E0000E36023189B7E1BB1E36843F48073E36037
:109E100023182044DA7E0F2A84BF0F22DA76C07E10
:109E2000E3681843E060FFF771FFE368E36110BD8A
:109E300078C6FF1F38B5C2001F4C111A214491F893
:109E4000213091F8205091F822101B0343EA85330A
:109E500043F46025012908BF2B46A2EB000108BF8F
:109E600043F480632144E56008BFE360E36891F850
:109E7000235091F8241043EA05230129E36004BF2D
:109E800043F08003E360131A2344121A93F8253039
:109E9000012B08BFE368224404BF43F04003E360A2
:109EA000E06892F8263040EA0310E060FFF72EFFEA
:109EB000E368A36238BD00BF78C6FF1F10B543003A
:109EC0001C4C1A18224492F92D103F29C4BF3F217F
:109ED00082F82D101A18224492F92D103F31BCBF80
:109EE000C12182F82D101A18224492F82E101F2931
:109EF00084BF1F2182F82E104FF44022E2601A180E
:109F00002244034492F82C202344012A04BF4FF436
:109F10005022E26093F82D00E26893F82E300002A0
:109F2000134300F4FE401843E060FFF7EFFEE368E0
:109F3000236310BD78C6FF1F10B58300244C1A1888
:109F4000224492F83410012984BF012182F8341090
:109F50001A18224492F83510032984BF032182F88D
:109F600035101A18224492F836100F2984BF0F2199
:109F700082F836101A18224492F83710032984BF49
:109F8000032182F837101A182244034492F838103B
:109F90000F29234484BF0F2182F8381093F838002A
:109FA00093F8342040F4202040EAC23093F8352062
:109FB00040EA423093F8362093F8373040EA0220E6
:109FC00040EA4310E060FFF7A1FEE368E36310BDE1
:109FD00078C6FF1F214B012010B503210024052264
:109FE00083F82C0083F825000220597283F8201092
:109FF00083F8211018729A72DC7283F82D2083F88E
:10A000002E2083F8224083F8234083F8244083F8ED
:10A01000260083F8344083F8354083F8364083F8CF
:10A02000374083F838405C769C76DC7618715C713A
:10A03000DC719C710A4B04229A602046FFF77CFF7A
:10A040002046FFF73BFF2046FFF7F4FE2046FFF7D0
:10A05000CDFE2046BDE810407CE600BF78C6FF1F5D
:10A06000C0F00F40044B042903EBC00318BF0022CB
:10A07000D97618BF5A76B9E678C6FF1F034B03EBB3
:10A08000C003597609B10422DA76AFE678C6FF1F1D
:10A09000024B03EBC0039976A8E600BF78C6FF1F0A
:10A0A000024B03EBC000C07E704700BF78C6FF1FA5
:10A0B000024B03EBC000407E704700BF78C6FF1F15
:10A0C000024B03EBC000807E704700BF78C6FF1FC5
:10A0D000024B03EBC00319713CE600BF78C6FF1FBB
:10A0E000024B03EBC003597134E600BF78C6FF1F73
:10A0F000024B03EBC003D9712CE600BF78C6FF1FEB
:10A10000024B03EBC003997124E600BF78C6FF1F22
:10A11000024B03EBC00319721CE600BF78C6FF1F99
:10A12000024B03EBC003597214E600BF78C6FF1F51
:10A13000024B03EBC00399720CE600BF78C6FF1F09
:10A14000024B03EBC0000079704700BF78C6FF1FC9
:10A15000024B03EBC0004079704700BF78C6FF1F79
:10A16000024B03EBC000C079704700BF78C6FF1FE9
:10A17000024B03EBC0008079704700BF78C6FF1F19
:10A18000024B03EBC000007A704700BF78C6FF1F88
:10A19000024B03EBC000407A704700BF78C6FF1F38
:10A1A000024B03EBC000807A704700BF78C6FF1FE8
:10A1B000034B00EB8002134483F83410BCE600BF6D
:10A1C00078C6FF1F034B00EB8002134483F8351061
:10A1D000B2E600BF78C6FF1F034B00EB80021344BA
:10A1E00083F83610A8E600BF78C6FF1F034B00EBCC
:10A1F0008002134483F837109EE600BF78C6FF1F25
:10A20000034B00EB8002134483F8381094E600BF40
:10A2100078C6FF1F034B00EB8000184490F8340011
:10A22000704700BF78C6FF1F034B00EB8000184447
:10A2300090F83500704700BF78C6FF1F034B00EB56
:10A240008000184490F83600704700BF78C6FF1FA2
:10A25000034B00EB8000184490F83700704700BFB4
:10A2600078C6FF1F034B00EB8000184490F83800BD
:10A27000704700BF78C6FF1F034B00EB400213443A
:10A2800083F82C101AE600BF78C6FF1F034B00EBC3
:10A290004002134483F82D1010E600BF78C6FF1F5C
:10A2A000034B00EB4002134483F82E1006E600BF78
:10A2B00078C6FF1F034B00EB4000184490F82C00B9
:10A2C000704700BF78C6FF1F034B00EB40001844E7
:10A2D00090F92D00704700BF78C6FF1F034B00EBBD
:10A2E0004000184490F82E00704700BF78C6FF1F4A
:10A2F000034BC0EBC002134483F820109AE500BF63
:10A3000078C6FF1F034BC0EBC002134483F8211033
:10A3100090E500BF78C6FF1F034BC0EBC00213449B
:10A3200083F8221086E500BF78C6FF1F034BC0EB01
:10A33000C002134483F823107CE500BF78C6FF1FDA
:10A34000034BC0EBC002134483F8241072E500BF36
:10A3500078C6FF1F034BC0EBC002134483F82510DF
:10A3600068E500BF78C6FF1F034BC0EBC002134473
:10A3700083F826105EE500BF78C6FF1F034BC0EBD5
:10A38000C000184490F82000704700BF78C6FF1F37
:10A39000034BC0EBC000184490F82100704700BF89
:10A3A00078C6FF1F034BC0EBC000184490F8220092
:10A3B000704700BF78C6FF1F034BC0EBC0001844B6
:10A3C00090F82300704700BF78C6FF1F034BC0EB17
:10A3D000C000184490F82400704700BF78C6FF1FE3
:10A3E000034BC0EBC000184490F82500704700BF35
:10A3F00078C6FF1F034BC0EBC000184490F826003E
:10A40000704700BF78C6FF1F2DE9F0479046334ADA
:10A41000089F099E1D461318044693F8403089464C
:10A420009246042B2FD8DFE803F0031A20262C00D5
:10A43000FFF790FC0AEB04030122C4EBC40454446C
:10A4400083F8402094F82630012B31D01FD3022B03
:10A4500035D016B1DAF800303370BDE8F087FFF779
:10A46000E9FC0AEB04030222E7E7FFF765FD0AEBCC
:10A4700004030322E1E7FFF721FD0AEB04030422B2
:10A48000DBE7FFF7B3FC0AEB04030022D5E7B9F1E1
:10A49000000F04D0DAF800309B0C89F80030B8F1D6
:10A4A000000FD6D0DAF800309B0A88F80030D0E7E9
:10A4B000002DCED0DAF800309B0A2B60C9E725B119
:10A4C000DAF80030DB0B5B012B60002FC1D0DAF82B
:10A4D0000030C3F384233B70BBE700BF78C6FF1F87
:10A4E00028B9034BDA7A12B90122DA7232E47047E2
:10A4F00078C6FF1F20B9034BD97A09B1D87229E475
:10A50000704700BF78C6FF1F062808D8DFE800F0B4
:10A5100004080B0E111417000A4B1B680B607047E0
:10A52000084BDB69FAE7074B1B69F7E7054BDB6B69
:10A53000F4E7044B1B6BF1E7024B9B6AEEE7014B20
:10A54000DB7AEBE778C6FF1F13B5C64C63789A1F1A
:10A55000012A0FD98C2B0DD0C02B0BD0C72B09D0C3
:10A5600003F16002D2B2182A04D903F13402D2B244
:10A57000322A05D8A27832B10422BB4B1A703BE1D3
:10A58000A278022AF8D8A42B00F05D8200F2A680FF
:10A59000842B00F03C8148D8062B00F00C8119D8A0
:10A5A000022B00F0348107D8002B00F01C81012B16
:10A5B00000F024810322E0E7042B23D040F2458100
:10A5C000D4F80310A078FFF746F9A378D4F8031065
:10A5D000A64A26E0802B00F006810ED80C2B00F056
:10A5E0004D810D2B00F06B81072BE3D1A278A04B9E
:10A5F00003EB4213E2789A72FEE0822B00F0748142
:10A6000040F2FC80A178D4F80320490141F0060112
:10A6100001F0E6010020FEF7EAFFA378D4F803106A
:10A62000944A42F8231000210CE1942B00F026817B
:10A6300028D88A2B00F061810ED8862BC0D0C0F0BC
:10A640000481872BB6D1A178D4F80320490141F0C9
:10A650000E0101F0EE0100E18D2B00F05C81932BE7
:10A6600000F02D818C2BA5D1E178A078C1F10801F3
:10A67000C9B2FFF7F7FCA2787D4B03EB4213E278F7
:10A68000DA72B9E0A02B00F0C9811BD8992B00F039
:10A690004E819A2B00F06781952B8BD1A1784901CF
:10A6A00041F0140101AA01F0F4010020FFF73FF886
:10A6B000D4F803209DF80530002A00F0358143F0DE
:10A6C0000403ECE0A22B00F0B78140F2AE81D4F895
:10A6D0000310A078C9B2FFF703FD8DE0B32B00F0A3
:10A6E00006823CD8AB2B00F0D1811CD8A72B00F000
:10A6F000B8810CD8A52B00F0AD81A62B7FF45AAF02
:10A70000D4F80310A078C9B2FFF70AFD74E0A92BB2
:10A7100000F0B58140F2AC81D4F80310A078C9B242
:10A72000FFF75AFD68E0AF2B00F0CC810BD8AD2BC2
:10A7300000F0C18140F2B181D4F80310A07849B291
:10A74000FFF7A4FD58E0B12B00F0CA8140F2C181AF
:10A75000D4F80310A078C9B2FFF7E8FD4CE0C32B92
:10A7600000F021811AD8B82B00F0DF810FD8B62B6A
:10A7700000F0C48100F2D181B52B7FF41BAFA27829
:10A780003B4B03EB4213D4F803209A6134E0C12B16
:10A7900000F0FB8000F20081C02B26E7D22B00F0F6
:10A7A00018810FD8CC2B00F00681D12B00F00B8143
:10A7B000C72B7FF4FFAEA2782D4B03EB4213E27858
:10A7C0005A7219E0D62B00F01781FE2B00F01C8185
:10A7D000D42B7FF4EFAEA278254B03EB4213D4F8D1
:10A7E00003205A6108E0A178D4F80320490101F060
:10A7F000E0010020FEF70DFF02B010BDA178D4F8F3
:10A800000320490141F0020101F0E201F1E7A178E2
:10A81000D4F80320490141F0080101F0E8010020CB
:10A82000FEF7E5FEA178D4F803204901002A41F0A3
:10A83000060101F0E601B8BF52420020FEF7D7FE44
:10A84000A37801210C4AD154D6E7A178D4F803208B
:10A85000490141F00A0101F0EA010020FEF7C7FEBC
:10A86000CAE700BFE4CEFF1F00D0FF1F0CD0FF1FC0
:10A87000C0CDFF1F18D4FF1FBCC6FF1FA178490120
:10A8800041F0140101AA01F0F4010020FEF74FFF8E
:10A89000D4F803209DF8053072B143F002038DF81F
:10A8A0000530A178490141F0140101AA01F0F40139
:10A8B0000020FEF777FE9FE723F00203EFE7A17881
:10A8C000490141F0140101AA01F0F4010020FEF752
:10A8D0002EFFD4F803209DF8053012B143F0010398
:10A8E000DDE723F00103DAE7A178D4F8032049017A
:10A8F00041F0040101F0E401AFE7A178490141F022
:10A90000140101AA01F0F4010020FEF710FFE37822
:10A910008DF80630C5E7A178D4F80320490141F04D
:10A920001A0101F0FA0198E723F00403B7E7A178D0
:10A93000490141F0180101AA01F0F8010020FEF7D9
:10A94000F6FE9DF80530E27823F00F0302F00F02C7
:10A950001343A1788DF80530490141F0180101AA8F
:10A9600001F0F801A4E7A178490141F0180101AA1A
:10A9700001F0F8010020FEF7DAFE9DF80530E278DC
:10A9800003F00F0343EA0213E3E7A2786A4B03EBF9
:10A990004213E2781A722FE7A378674AD4F80310BB
:10A9A0005B01D15028E7A278634B03EB4213D4F844
:10A9B00003205A6020E7A2785F4B03EB4213D4F8E0
:10A9C0000320DA8118E7D4F80310A07804F07EF8A9
:10A9D00012E7A078584BE178D4F8032003EB40133A
:10A9E00001F01F011A6104F061F8D4F80310A07897
:10A9F000491104F053F8FFE6A2784F4B03EB4213E2
:10AA0000D4F803209A83F7E64B4BA178D4F80320BF
:10AA100003EB411302B101221A73EDE6D4F80310DF
:10AA2000A078C9B2FFF72AFBE6E6D4F80310A078B5
:10AA3000C9B2FFF72DFBDFE6D4F80310A078C9B246
:10AA4000FFF746FBD8E6D4F80310A078C9B2FFF7A9
:10AA500057FBD1E6D4F80310A078C9B2FFF758FB32
:10AA6000CAE6D4F80310A078C9B2FFF761FBC3E6C9
:10AA7000D4F80310A078C9B2FFF79AFBBCE6D4F86B
:10AA80000310A078C9B2FFF79DFBB5E6D4F8031018
:10AA9000A078C9B2FFF7AAFBAEE6D4F80310A078FD
:10AAA000C9B2FFF7ADFBA278244B03EBC203D4F885
:10AAB00003205A71A0E6D4F80310A078C9B2FFF7BA
:10AAC000DBFB99E6D4F80310A078C9B2FFF710FCBD
:10AAD00092E6D4F80310A078C9B2FFF713FC8BE616
:10AAE000D4F80310A078C9B2FFF716FC84E6D4F8B6
:10AAF0000310A078C9B2FFF72DFC7DE6A078D4F84A
:10AB000003200E4B43F83020002A7FF475AE03EB90
:10AB1000C0035979FFF774FB6EE6A278074B03EB8D
:10AB2000C203D4F803201A7166E6D4F80310A078A3
:10AB3000C9B2FFF7DDFA5FE6C0CDFF1F34CDFF1FBE
:10AB400037B5C44DC44C6B789A1F012A0FD98C2B92
:10AB50000DD0C02B0BD0C72B09D003F16002D2B2AD
:10AB6000182A04D903F13402D2B2322A05D8AA78BD
:10AB700032B10423237003B030BDAA78022AF8D87A
:10AB8000A32B00F0348200F2C180832B00F0778188
:10AB90005CD8082B00F0A7801ED8032B00F068813A
:10ABA0000ED8012B00F04F8140F24481A978490171
:10ABB00041F0080101F0E8010020FEF7CFFD40E17F
:10ABC000052B4FD0C0F05B81062B00F05D81072B79
:10ABD00000F071810323A5E10C2B00F0728114D8E1
:10ABE0000A2B00F0848140F27B8101AA7C210020A5
:10ABF000FEF79DFDAB785A00022393409DF8062096
:10AC0000134214BF0123002343E1802B00F0128183
:10AC100010D80D2BDED1A978490141F0140101AA09
:10AC200001F0F4010020FEF782FD9DF8053003F0ED
:10AC300001032EE1812B00F00681822BCAD1A97875
:10AC4000490141F0040101F0E401B5E7942B00F063
:10AC5000388122D8872B00F0558106D8852B00F04B
:10AC60000781A3D9AA787D4B0BE18C2B00F0518191
:10AC70000ED88A2BAED1A978490141F0140101AA5E
:10AC800001F0F4010020FEF752FD9DF8063000E1CE
:10AC90008D2B00F04981932BBCE79C2B00F0278182
:10ACA0001AD8992B00F0478110D8952B92D1A9780A
:10ACB000490141F0140101AA01F0F4010020FEF75E
:10ACC00036FD9DF80530C3F38003E2E09A2B00F0D7
:10ACD00041819B2B89D07DE7A02B00F080810BD890
:10ACE0009D2B7FF477AF0020FEF71BFDAB785B0058
:10ACF000184100F00100A4E0A12B00F07481A22B08
:10AD00007FF468AFA878FFF71BFA9AE0B52B00F044
:10AD1000A8813AD8AC2B00F086811BD8A72B00F075
:10AD2000728108D8A52B00F06A8140F26481A8786E
:10AD3000FFF72EFA85E0A92B00F06D81C0F0678146
:10AD4000AA2B00F06C81AB2B7FF444AFA878FFF7FF
:10AD50007FFA76E0B02B00F0748108D8AE2B00F0BB
:10AD60006C8140F26681A878FFF708FB69E0B22B9E
:10AD700000F06F81C0F06981B32B00F06E81B42BBD
:10AD80007FF428AFAB78364A39E0C72B7CD01DD88A
:10AD9000C02B00F090800BD8B72B00F06D81C0F075
:10ADA0006681B82B7FF416AFA878FFF7D9F948E091
:10ADB000C22B00F0E380C0F0DB80C32B00F0E38007
:10ADC000C42B7FF407AFAA78264B5AE0D12B00F0B2
:10ADD000F68016D8CE2B00F0DC8008D8CC2B7FF480
:10ADE000F9AEAA78204B03EB4213DB8951E0CF2B5D
:10ADF00000F0D280D02B7FF4EDAEAB781B4AD35C51
:10AE000047E0D42B00F0DF8008D8D22B7FF4E2AEED
:10AE1000AA78154B03EB42131B693AE0D62B00F0DE
:10AE2000D880FE2B7FF4D6AEAA780F4B03EB4213EB
:10AE30001B7B2EE0A978490101F0E0010020FEF71C
:10AE400095FE606026E0A978490141F0020101F019
:10AE5000E201F3E7E4CEFF1F00D0FF1F0CD0FF1F7D
:10AE600030CDFF1F1CCDFF1FC0CDFF1FBBCDFF1F6F
:10AE7000A978490141F00A0101F0EA019CE6AA78AB
:10AE8000824B53F8223004E0AA78814B03EB421343
:10AE90005B7A63607F4B1B78002B3FF46CAE7E4B7C
:10AEA00062681A607D4B002A40F0EC801A6842F01C
:10AEB00008021A605FE6AA78754B03EB42139B7A8F
:10AEC000E7E7A978490141F0140101AA01F0F40172
:10AED0000020FEF72CFC9DF80530C3F34003D8E7B3
:10AEE0000020FDF72CFE003018BF0120A9E701AAC1
:10AEF0007C210020FEF71BFCAA789DF8063052004A
:10AF0000134194E6A978490141F00E0101F0EE01E8
:10AF100052E6AB782BB90020FFF7C2F8C0F1080069
:10AF20008FE704232370B5E7A978490141F01A019E
:10AF300001F0FA0140E6A978490141F0180101AA9F
:10AF400001F0F8010020FEF7F2FB9DF8053003F058
:10AF50000F039EE7A978490141F0180101AA01F009
:10AF6000F8010020FEF7E3FB9DF805301B0990E790
:10AF7000AA78474B03EB42131B7A8AE7AB78444A23
:10AF80005B01D35885E7AA78414B03EB42135B681A
:10AF90007FE7AA78424B74E7AB78424AD05C002145
:10AFA000616008B101206060D1543F4AD15C19B1A1
:10AFB000616841F0020161600021D1546AE7A8781C
:10AFC00003F078FD3DE7AA78314B03EB42135B6950
:10AFD0005FE7AA782E4B03EB42139B8B59E7A878C7
:10AFE000FFF766F82DE7A878FFF76AF829E7A87851
:10AFF000FFF7AEF825E7A878FFF7BAF821E7A878B9
:10B00000FFF7BEF81DE7A878FFF7CAF819E7A87898
:10B01000FFF700F915E7A878FFF706F911E7A87818
:10B02000FFF70CF90DE7AA78204B03EBC2035B791D
:10B030002FE7A878FFF73EF903E7A878FFF744F970
:10B04000FFE6A878FFF7A4F9FBE6A878FFF7AAF9CE
:10B05000F7E6A878FFF7B0F9F3E6A878FFF7C0F9AC
:10B06000EFE6AA780A4B03EB42139B6911E7AA7833
:10B070000E4B53F832300CE7AA780C4B03EBC203AB
:10B080001B7906E71A6822F0080212E718D4FF1F9E
:10B09000C0CDFF1FFBCFFF1FECCFFF1FECCEFF1F6C
:10B0A00054CDFF1FB8CDFF1F4FCDFF1F34CDFF1F65
:10B0B00038B5984A9378022B144600F02481032B6C
:10B0C00000F03681002B40F0098253784E2B00F0BF
:10B0D000C18031D8462B00F08F8012D8422B7BD014
:10B0E00006D8402B6CD0412B71D003228A4B65E0EF
:10B0F000442B76D0452BF8D1884BD1785971052057
:10B1000061E04B2B00F096800CD8472B7CD0492B6C
:10B11000EBD1D278814B002A40F08780DA75D97D57
:10B12000172050E04C2B00F090804D2BDDD17B4B55
:10B13000D1785975152046E0542B00F0BD801BD8FE
:10B14000512B00F0A48009D84F2B00F08E80502B9B
:10B15000CBD1724BD1789975162034E0522B00F088
:10B16000A380532BC1D16D4DD2F803302946042260
:10B1700041F8103F10204FE0832B00F0B58014D829
:10B18000552B00F0A580562BAFD1D2F803300F2BF2
:10B1900000F2A481D1780020FEF73CFB5F49E37800
:10B1A00001F8243F0122242022E0852B00F0A68014
:10B1B000C0F09F80FF2B98D1D278594B1A7038BDC0
:10B1C000D17840F2FF70BDE83840FDF7B5BF534B72
:10B1D000D17819700020F6E7504BD17859700120D2
:10B1E000F1E74E49D2F8033041F81C3F04221C20FD
:10B1F000BDE83840FDF7FFBF4849D2F8033041F8B9
:10B200000C3F04220C20F3E7444DD2F803302946CA
:10B21000042241F8083F0820FDF7EDFF2A8A29891A
:10B220006879BDE8384003F089BA3B490122DA75F4
:10B230004A6074E7394CD178E1700320FDF77CFF58
:10B24000E078BDE83840FDF7DBBA344BD17899702F
:10B250000220B8E7314CD2F80300E084FDF7EBFCA4
:10B26000022204F126012620C2E7D2F803102B4C5B
:10B27000C9B219206176FDF75FFF617E11F001010F
:10B2800018BF01210020BDE83840FEF7ABBC234DBC
:10B290002A7DD20704D5E378DB0701D4FDF7B3FE9E
:10B2A000E178297514208EE71C49D2F8033041F863
:10B2B000203F042220209BE7D2F80330012B00F22C
:10B2C0000D811649D37801F81A3F01221A208FE721
:10B2D000D2F80330012B00F201811049D37801F834
:10B2E0001B3F01221B2083E70E4BD2F803205A603C
:10B2F00038BD0D4BD2F803201A6038BD094BD2F887
:10B3000003209A6038BD5178084BD2F8032043F8E7
:10B31000212038BDE4CEFF1F00D0FF1F0CC0FF1F4F
:10B32000FACFFF1FBCC6FF1FFCCFFF1F18D0FF1FA7
:10B3300053782E2B3FF6D9AE01A252F823F000BF6E
:10B34000FDB300000FB4000021B40000EBB000001A
:10B35000EBB00000EBB00000EBB00000EBB0000081
:10B36000EBB0000033B400003DB4000047B400006F
:10B37000EBB00000EBB00000EBB00000EBB0000061
:10B38000EBB00000EBB00000EBB00000EBB0000051
:10B39000EBB00000EBB00000EBB00000EBB0000041
:10B3A000EBB00000EBB00000EBB0000051B40000C7
:10B3B0005FB400006DB4000075B400007DB40000FF
:10B3C00085B40000EBB00000EBB00000EBB0000073
:10B3D000EBB00000EBB00000EBB000008DB400005B
:10B3E00097B40000A1B40000ABB40000B5B40000F5
:10B3F000BFB40000C9B40000D3B40000384BD4F887
:10B4000003201A60FDF786F9364BD86038BD344BFF
:10B41000D4F803205A60FDF77DF9324B186138BD2E
:10B420002F4BD4F803209A60FDF774F92D4B586127
:10B4300038BD2B4BD4F80320DA6038BD284BD4F844
:10B4400003201A6138BD264BD4F803205A6138BD59
:10B45000D4F803100020BDE83840FEF7E6BAD4F86F
:10B4600003100020BDE83840FEF709BBD4F80310F4
:10B470000120F0E7D4F803100120F3E7D4F803101B
:10B480000220E8E7D4F803100220EBE7144BD4F8CD
:10B4900003209A6138BD124BD4F80320DA6138BD1D
:10B4A0000F4BD4F803201A6238BD0D4BD4F803209B
:10B4B0005A6238BD0A4BD4F803209A6238BD084B53
:10B4C000D4F80320DA6238BD054BD4F803201A63A0
:10B4D00038BD034BD4F803205A6338BD042205E677
:10B4E00030CEFF1FBCC6FF1F2DE9F0478046164631
:10B4F0000F4600294BD0002849D0814247D0540143
:10B5000064B244F00605EDB229460020FEF72EFB9A
:10B5100044F00C0101F0EC0182460020FEF726FB0E
:10B520008146404605F0F0FF0446384605F0ECFF42
:10B530000146204606F0F4F80746504605F0E4FFC1
:10B54000394606F0EDF806F0FDF90446484605F0E8
:10B55000DBFF394606F0E4F806F0F4F9002C08BFEA
:10B5600001240C49002814BF80464FF001083846DA
:10B5700006F0C0F918B141463046FEF76CF9224694
:10B5800029460020FEF745F8034B01229A55BDE8F5
:10B59000F08700BF0000A041BCC6FF1F70B50C4D76
:10B5A0002B5C04469BB1C6B20A4B710141F0060107
:10B5B00053F8202001F0E6010020FEF718F8064BB2
:10B5C000304653F82410FEF746F900232B5570BD82
:10B5D000BCC6FF1F18D4FF1F0CD0FF1F2DE9F04F72
:10B5E000C44EC54F32787A7064233B70212AD6F856
:10B5F00003307B6085B034463D4601F0ED8200F2B9
:10B60000C1800E2A00F0A48739D8072A00F0AB8346
:10B6100014D8032A00F0EE8108D8012A00F099819D
:10B62000022A00F0BF8102232B70B8E1052A00F046
:10B63000978340F2FB81FFF783FAB0E10A2A00F01A
:10B64000B88507D8082A00F07484092AEBD1FFF7DF
:10B650002FFDA4E10C2A00F0488740F22E87B07835
:10B66000022800F291837378012B00F05687C0F016
:10B670005087022B00F0558703233B708FE1182A77
:10B6800001F0B1802BD8142A01F0058015D80F2ABB
:10B6900000F08787132AC6D17178984A092900F2E9
:10B6A000CE87DFE811F0C907D507D807DB07DF072A
:10B6B000E607E907EC07EF07E407162A01F08F8099
:10B6C00041F20A808E4A116A072900F26881481CFB
:10B6D00002EB81011062D0694862D3615FE11C2AEC
:10B6E00001F0858120D81A2A01F09B8041F28880E0
:10B6F000834D95F8452062B95E1C04BF7F4B1B68E3
:10B700000A205843A864FDF705F80123E86485F88A
:10B7100045306378042B00F24281DFE813F0930890
:10B72000D90806093709B1081F2A01F0948101F2EE
:10B73000E4811E2A7FF477AF7278142A00F2CD8656
:10B74000B078022801F2588102EB42046D4D0444A6
:10B7500045F824306C4B9B7E002B00F02081002AA2
:10B7600000F01D81032111FB02010C23013A5A4311
:10B7700002F5C363042205EB810102FB0030FDF7F3
:10B780003AFD0CE1802A01F0008344D8402A01F000
:10B79000E48229D8242A01F07D820CD8222A01F0E3
:10B7A0007182232A7FF43FAF544B1B68C6F80330E5
:10B7B000FFF77EFCF3E0262A01F0A982C1F09D820A
:10B7C000272A7FF430AFB278022A00F2DD82737844
:10B7D000142B00F2828603EB43031344474A11689B
:10B7E000484A42F82310DAE0442A01F0C28207D81E
:10B7F000422A01F0BA8241F2B48202F038F9CEE076
:10B80000462A01F0BE82C1F0B882472A7FF40BAF0E
:10B8100002F031F9C3E0872A01F05A8346D8832A1F
:10B8200001F0CF8209D8812A01F0B482822A7FF404
:10B83000FAAE334B02221A76B1E0852A01F0F38288
:10B84000314A41F2DD823149314C01250D70917848
:10B85000217040F2FE718B4201F2EA82127D12EAFF
:10B86000050641F0E582184601A9FDF78BFB9DF81E
:10B87000043063709DF80530A3709DF80630E370C6
:10B880009DF80A3023719DF8093063719DF80830E6
:10B89000A3719DF80730E37126722B46E15C227A92
:10B8A00001330A44082B2272F8D178E08C2A01F087
:10B8B00055833BD8892A01F03683C1F0D1828A2A88
:10B8C0007FF4B1AE7278134B002A41F044831A70B2
:10B8D000114AE37813700A4A92F834110F4A117032
:10B8E0000F4900220A700F490A700F4A11780B4362
:10B8F000137054E0E4CEFF1F00D0FF1FECCFFF1FFA
:10B90000BCC6FF1FF0CEFF1F0CC0FF1FF0CFFF1FF4
:10B91000F1CFFF1F28CDFF1F53CDFF1F78CEFF1F94
:10B9200052CDFF1FB1CEFF1F29CDFF1FF22A01F01C
:10B930008583FF2A01F0C7838D2A7FF474AE727865
:10B94000032A01F27783DFE812F04A0B310B630B15
:10B95000710BB178022900F21782C64B01225A54AA
:10B96000C54B00255D54C54B022228465D54FDF7AA
:10B970000BFFB178490141F0060140F2FF7201F07E
:10B98000E6012846FDF733FEB178D6F803204901D9
:10B9900041F0080101F0E8012846FDF728FE05B056
:10B9A000BDE8F08FB178022900F2EE81B14B01229F
:10B9B0005A54B14B00255D54B04B284602225D54C9
:10B9C000FDF7E2FEB178490141F00601284640F258
:10B9D000FF7201F0E601FDF70AFEB178D6F8032008
:10B9E000490141F00801524201F0E8012846FDF703
:10B9F000FEFDD4E7B078022800F2C68102F01AFEFC
:10BA00000222B1780020FDF7BFFEB178490141F074
:10BA1000080101F0E8010020FDF76CFEB378954ABB
:10BA20000121D154954A0021D154B8E7B0780228B9
:10BA300003D97278022A40F0A7816278032A00F2C3
:10BA40008C81DFE812F0040022004C005601FFF761
:10BA5000A5FDA178894B8A4800255D54864B5D542D
:10BA6000012303FA01F20378490123EA0203037078
:10BA7000D4F80320284601F0E001FDF7CAFD2A466C
:10BA8000A1782846FDF780FE89E7FFF787FDA178BA
:10BA90007A4B00265E54784B5E54490141F0020116
:10BAA00001F0E2013046FEF761F8D4F80370A178A6
:10BAB00007447348012303FA01F20378490123EA9A
:10BAC000020303703A4601F0E0013046FDF7A1FDA4
:10BAD0003246A1783046FDF757FE6F605FE7142BC2
:10BAE00000F3528110F0C00624D1022800F24C81EC
:10BAF00003EB43030344634A614D52F82370FFF79D
:10BB00004DFDA1785D4B5E545B4B5E54012303FAFF
:10BB100001F02B78490123EA00033A46304601F050
:10BB2000E0012B70FDF775FD3246A1783046FDF738
:10BB30002BFE34E7402E40F0A780002601960296A7
:10BB40000396324640FA02F1C90706D504A93144EA
:10BB50000136032E01F8102C02D00132032AF1D154
:10BB6000DFF82081002703EB4309B7423DD1012FC5
:10BB70000BDD022F019E029D55D1AE424EDD9DF898
:10BB8000012029463046FFF7AFFC3E4FDFF8EC803E
:10BB9000DFF8E4900025A3782B41DA0721D5D4F80B
:10BBA0000330374803EB43032B445FFA85FA57F819
:10BBB0002320012303FA05F10378002623EA010379
:10BBC0004FEA4A11037001F0E001304605F80860C1
:10BBD00005F80960FDF71DFD324651463046FDF778
:10BBE000D3FD0135032DD6D1D9E61DF807502846DF
:10BBF000FFF7D4FC690141F0020101F0E2010020ED
:10BC00004D44FDF7B3FF58F82520801A002801ABFA
:10BC1000B8BF404243F827000137A6E79DF800204F
:10BC200031462846AFE7AE42039F16DDBE4209DD2E
:10BC30009DF8012029463046FFF756FC9DF802206A
:10BC400039469FE79DF8002031463846FFF74CFC07
:10BC50009DF801202946384695E7BD4231469DF8BA
:10BC60000020F2DD2846FFF73FFC9DF80220394610
:10BC7000D7E700BFBCC6FF1FB8CDFF1F4FCDFF1FCA
:10BC800029CDFF1FF0CEFF1F802E7DD1DFF8F89267
:10BC9000BB4FDFF8F8820025A3782B41DB0724D5C2
:10BCA000D4F8033003EB43032B44284659F823A070
:10BCB000FFF774FCB34A012303FA05F113785FFA26
:10BCC00085FB002623EA01034FEA4B11137001F0B4
:10BCD000E00152463046EE5505F80860FDF799FC44
:10BCE000324659463046FDF74FFD0135032DD3D17D
:10BCF00055E6022848D8142B46DC400140F00201EA
:10BD000001F0E2010020FDF731FFD4F80330A17803
:10BD10009D4A03EB43030B44002652F8235005448D
:10BD20000846FFF73BFCA178954B96485E54974B2D
:10BD30005E54012303FA01F20378490123EA020366
:10BD400003702A46304601F0E001FDF762FC3246FE
:10BD5000A1783046FDF718FD21E603232B701EE67F
:10BD6000FEF7F2FB1BE673789A1F012A0AD98C2B87
:10BD700008D0C02B06D0C72B04D003F13402D2B2B6
:10BD8000322A04D8A2782AB104232B7007E6B278AD
:10BD9000022AF9D8952B2BD8932B71D20D2B17D8BB
:10BDA0000C2B6DD2052B5CD004D8042B54D003236C
:10BDB0002B70F4E5062B59D0072BF8D1A078744BE3
:10BDC00003EB40134001997A4A30FDF7B5F9E6E5F7
:10BDD000862B46D003D8822B57D0832BE6E78C2BBB
:10BDE00058D08D2BE3D11A21A078FDF7E5FDD6E5DB
:10BDF000C32B76D00FD8B52B56D007D8993B012B43
:10BE0000D5D81821A078FDF7D7FDC8E5C12B55D0AE
:10BE10005ED8C02BD1E7D22B6DD00DD8C72B25D043
:10BE2000CC2BC4D1A0785B490230400101440222EE
:10BE30000E30FDF7E0F9B2E5D62B66D0FE2B6ED0C2
:10BE4000D42BB4D1A07854490230400101440422DB
:10BE50001430FDF7D0F9A2E50621A078FDF7ACFD7E
:10BE60009DE50C21A078FDF7A7FD98E5A078484B4B
:10BE700003EB40134001597A4930FDF75DF98EE537
:10BE80001421A078FDF798FD89E50421A078FDF73D
:10BE900093FD84E5A378002B7FF476AF01223F4920
:10BEA0004B20FDF7A8F97AE5A0783D490230400122
:10BEB000014404221830FDF79EF970E5A078344B58
:10BEC00003EB40134001197A4830FDF735F966E578
:10BED000A07834490230400104220144FDF78BF977
:10BEE0005DE5A0783049023040010422014410444D
:10BEF000FDF781F953E5A0782C4902304001014457
:10BF000004221030FDF777F949E5A078284902307E
:10BF10004001014402221C30FDF76DF93FE5A07895
:10BF2000244902304001014401220C30FDF763F93D
:10BF300035E573789A1F012A0AD98C2B08D0C02BBB
:10BF400006D0C72B04D003F13402D2B2322A33D840
:10BF5000A278002A7FF418AF952B52D8932B80F04B
:10BF6000C3800D2B3BD80C2B80F0BE80052B00F03E
:10BF7000988025D8042B7FD003232B700FE500BFBA
:10BF80004FCDFF1F29CDFF1FF0CEFF1FB8CDFF1FE4
:10BF9000C0CDFF1F8ECDFF1F94CDFF1FCBCDFF1F48
:10BFA00098CDFF1F80CDFF1F84CDFF1F90CDFF1FB9
:10BFB0009CCDFF1F8CCDFF1FB278022ACCD9E3E6BF
:10BFC000062B00F08780072BD6D1A47860014A3079
:10BFD000FDF78BF9B54B03EB44139872DFE4862B26
:10BFE0005FD004D8822B00F08480832BC3E78C2B96
:10BFF00000F084808D2BBFD11A21A078FDF7B8FC0A
:10C00000CDE4C32B00F0AC8012D8B52B00F08B80B0
:10C0100007D8993B012BAFD81821A078FDF7A8FCD1
:10C02000BDE4C12B00F0898000F29180C02BCBE7EA
:10C03000D22B00F09F800DD8C72B4BD0CC2B9BD19F
:10C04000A0789B4902304001014402220E30FDF7E6
:10C0500065F9A4E4D62B00F09780FE2B00F09E80BB
:10C06000D42B89D1A07893490230400101440422A5
:10C070001430FDF753F992E40621A078FDF778FC1F
:10C08000A578690141F0060101F0E6010020FDF705
:10C0900065FB894B894A43F82500A3780021D154D8
:10C0A0007DE4A0780C21FDF763FCA578690141F0DF
:10C0B0000C0101F0EC010020FDF750FB804B7F4AA2
:10C0C00043F82500A0780021115453F82010FDF703
:10C0D000C2FB64E4A47860014930FDF706F9734BB4
:10C0E00003EB441358725AE41421A078FDF740FC86
:10C0F00055E40421A078FDF73BFC50E4A378002B25
:10C100007FF442AE694D012205F10B014B20FDF792
:10C1100005F9A07805EB4015E97AC1F10801C9B22B
:10C12000FDF7A0FF3BE4A0786649023040010144DE
:10C1300004221830FDF7F2F831E4A47860014830A9
:10C14000FDF7D3F8594B03EB4413187227E4A0789A
:10C150005D490230400104220144FDF7DFF81EE48E
:10C16000A0785A4902304001042201441044FDF7EE
:10C17000D5F814E4A0785649023040010144042265
:10C180001030FDF7CBF80AE4A078524902304001A4
:10C19000014402221C30FDF7C1F800E4A0784E49AA
:10C1A00002304001014401220C30FDF7B7F8FFF7DF
:10C1B000F6BBB378022B00F0DA80032B00F0DC80B2
:10C1C000002B40F072817378502B00F0A78027D8A5
:10C1D000472B00F0938012D8422B64D006D8402B16
:10C1E00046D0412B5BD003232B7046E0452B7FD0FC
:10C1F00000F28180442BF6D1384BDB6951E04C2BA7
:10C2000000F0858006D8492B7BD04B2BEBD1334BEC
:10C21000DB7846E04E2B314B7ED07BD95B7E40E015
:10C22000802B00F08A8012D8532B7DD006D8512B5A
:10C2300077D0522BD7D1294B1B6A32E0552B79D0BE
:10C2400075D3562BCFD1254B93F8243029E0832B7F
:10C250007CD005D8812B73D0822BC4D1174BCCE76F
:10C26000852B79D075D3FF2BBDD11D4B1B784AE0B0
:10C2700040F2FF70FDF739F868601A4B1B78002B0D
:10C280003FF48DAB184B6A681A60184B002A40F0D7
:10C290000E811A6842F008021A60FFF780BB0F4B4C
:10C2A0001B786B60E9E70D4B5B78FAE7C0CDFF1FA9
:10C2B0008ECDFF1F94CDFF1F18D4FF1FBCC6FF1FDC
:10C2C0000CD0FF1F98CDFF1F80CDFF1F84CDFF1F17
:10C2D00090CDFF1F9CCDFF1F8CCDFF1F0CC0FF1FFB
:10C2E000FACFFF1FFBCFFF1FECCFFF1FECCEFF1FCE
:10C2F000B04B5B79D5E7AF4BDB68D2E7AD4B9B68C2
:10C30000CFE7AC4BDB7D003318BF0123C9E7A94B56
:10C310009B78C6E75B7DC4E7DB8CC2E7A54B9B7DC2
:10C32000BFE7A44B1B7DBCE7A24B1B69B9E7A14B40
:10C330009B7EB6E79F4BDB7EB3E79F4B1B7EB0E750
:10C340009D4B1B7E1E1F73427341AAE79A4B5B688D
:10C35000A7E79A4B1B68A4E7974A9948936843F26A
:10C36000390100FB0313936023F0004399E77278CF
:10C37000944B53F8223094E773782E2B3FF633AF6B
:10C3800001A252F823F000BF45C4000049C40000D8
:10C390004DC40000E7C10000E7C10000E7C1000094
:10C3A000E7C10000E7C10000E7C1000051C4000080
:10C3B00055C4000059C40000E7C10000E7C10000F7
:10C3C000E7C10000E7C10000E7C10000E7C10000CD
:10C3D000E7C10000E7C10000E7C10000E7C10000BD
:10C3E000E7C10000E7C10000E7C10000E7C10000AD
:10C3F000E7C100005FC4000067C400006FC4000014
:10C4000073C4000077C400007BC40000E7C10000D3
:10C41000E7C10000E7C10000E7C10000E7C100007C
:10C42000E7C100007FC4000085C4000089C400008B
:10C430008DC4000093C4000099C400009FC4000094
:10C44000A5C40000604B85E75F4B80E75E4B56E775
:10C450005D4B51E75C4B68E75B4B5B6921E7002074
:10C46000FDF737FB08E70020FDF748FB04E7012054
:10C47000F6E70120F8E70220F2E70220F4E7524B4A
:10C480009B690EE7504BB8E64F4BD5E64E4B5B6AC7
:10C4900007E74D4B9B6A04E74B4BDB6A01E74A4BCE
:10C4A0001B6BFEE6484B5B6BFBE604239CE61A68BD
:10C4B00022F008021A60FFF772BAB378022B10D18B
:10C4C0007078372809D800F5A77040498000042209
:10C4D0000144FCF790FEFFF762BA03232B70FFF7CD
:10C4E0005EBA04233B70FFF75ABAB378022B0CD123
:10C4F00070783728F1D800F5A770344980000422FD
:10C500000144FCF70BFFFFF74ABA04233B70FFF727
:10C5100046BA02F087F8FFF742BA02F08BF8FFF74D
:10C520003EBA02F08FF82A4B78601B78002B3FF45C
:10C5300036AA284B1860284B1A6820B942F0080226
:10C540001A60FFF72CBA22F008021A60FFF727BA28
:10C55000B2782AB1022A0CD004233B70FFF71FBA2D
:10C560007278002A7FF41BAA1846FCF7CDFBFFF770
:10C5700016BA7078072808D81BB9FCF7ABFAFFF792
:10C580000EBAFCF783FAFFF70ABAFF287FF407AA6E
:10C590005D1C0ABF0F4BD8B21878FCF7BFFAFFF743
:10C5A000FEB9B378012B39D0C3B1022B3AD00423A2
:10C5B0003B701EE00CC0FF1FBCC6FF1FFCCFFF1F5F
:10C5C0006D4EC64118D0FF1F30CEFF1FE0CAFF1FBF
:10C5D000FBCFFF1FECCFFF1FECCEFF1F70780828AA
:10C5E00003D8FCF7ACFA686003E00A2811D10023F5
:10C5F0007B609E4B1B78002B3FF4D1A99C4B6A6853
:10C600001A609C4B92B91A6842F008021A60FFF750
:10C61000C6B9FF28EDD1FCF7FDFAE4E7707802F027
:10C620005BF8E0E77078FCF7BFFADCE71A6822F005
:10C6300008021A60FFF7B3B9106818441060126856
:10C640008C4B12BB1A6842F008021A60FFF7A7B9B8
:10C650001068C01AF2E710685843EFE7106890FBC3
:10C66000F3F0EBE7116891FBF3F003FB1013136099
:10C67000E5E710681840E1E710681843DEE7106846
:10C680005840DBE71368DB43F1E71A6822F0080241
:10C690001A60FFF784B9764A1168764A8B421368AC
:10C6A0000BDA23F0030343F004031360136871B93A
:10C6B00043F008031360FFF772B90BBF23F00603C2
:10C6C00023F0050343F0010343F00203EDE723F0F9
:10C6D00008031360FFF763B972780C2A3FF65FA96D
:10C6E000DFE802F0071019222B343E475059626BE5
:10C6F0007400604A126814077FF551A95E4AD3613D
:10C70000FFF74DB95B4A126810073FF548A95A4A2E
:10C71000D361FFF744B9574A1268D1077FF53FA9A3
:10C72000554AD361FFF73BB9524A1268D2073FF529
:10C7300036A9514AD361FFF732B94E4A12685707FA
:10C740007FF52DA94C4AD361FFF729B9494A1268F0
:10C7500012F0050F3FF423A9474AD361FFF71FB931
:10C76000444A126896077FF51AA9434AD361FFF736
:10C7700016B9404A126895073FF411A93E4AD361A1
:10C78000FFF70DB93B4A1268D4067FF508A93A4A6B
:10C79000D361FFF704B9374A126890067FF5FFA806
:10C7A000354AD361FFF7FBB8324A126851067FF56C
:10C7B000F6A8314AD361FFF7F2B82E4A1268120682
:10C7C0007FF5EDA82C4AD361FFF7E9B8294A126832
:10C7D000D7057FF5E4A8284AD361FFF7E0B8264AD9
:10C7E000D361FFF7DCB8244A136A002B3FF4D7A8C3
:10C7F000013B136202EB83035B6AD361FFF7CFB89F
:10C8000073782E2B04D81D4A0121D154FFF7C7B8E5
:10C81000FF2B7FF462AE184B012283F84420FFF710
:10C82000BEB873782E2B04D8144A0021D154FFF7D8
:10C83000B6B8FF2B7FF451AE0F4B002283F8442093
:10C84000FFF7ADB8FBF766FFEB6CC01A0028AB6CC6
:10C85000B8BF4042984295BFEB69002303F1FF3314
:10C8600085F8453098BFEB61FFF799B8FBCFFF1F04
:10C87000ECCFFF1FECCEFF1FBCC6FF1F82CEFF1FF9
:10C88000A07801F0DFFE40B9B74A85F8450013688B
:10C8900023F010031360FFF782B8AB6C9BB1FBF77A
:10C8A00039FFEB6CC01A0028AB6CB8BF404298420D
:10C8B00009D9AD4A002385F84530136843F01003C9
:10C8C0001360FFF76CB8EB69013BEB61FFF767B8EA
:10C8D0000020FCF726FFA3785B00184110F001044C
:10C8E00009D0A14A002385F84530136823F01003CE
:10C8F0001360FFF754B8AB6C93B1FBF70BFFEB6C15
:10C90000C01A0028AB6CB8BF4042984208D9964A7A
:10C9100085F84540136843F010031360FFF73FB8F4
:10C92000EB69013BEB61FFF73AB801AA7C210020DB
:10C93000FCF7FDFEA3789DF806405A0002239340C1
:10C940001C4009D0884A002385F84530136823F03D
:10C9500010031360FFF723B8AB6C93B1FBF7DAFE5B
:10C96000EB6CC01A0028AB6CB8BF4042984208D9A3
:10C970007D4A85F84540136843F010031360FFF7C4
:10C980000EB8EB69013BEB61FFF709B801AA7C2106
:10C990000020FCF7CCFEA2789DF80630520013412F
:10C9A00013F0010409D0704A002385F8453013685C
:10C9B00023F010031360FEF7F2BFAB6C93B1FBF7EB
:10C9C000A9FEEB6CC01A0028AB6CB8BF404298427D
:10C9D00008D9654A85F84540136843F01003136091
:10C9E000FEF7DDBFEB69013BEB61FEF7D8BF5F4BA4
:10C9F00000221A76FEF7D3BFFF287FF4C5A95C4E4C
:10CA00003AB300254FF003080C27607818FB00515B
:10CA10000138784300F5C36000EB8500042206EB83
:10CA200081010135FCF7E7FB032DEED1FEF7B7BF1F
:10CA300061197819042231440435FCF7DCFB0C2D14
:10CA4000F6D10C34FC2C3EF4AAAF002504F20C679E
:10CA5000EEE70C24F9E77378142B3FF63EADB2787D
:10CA6000022A1BD803EB43031344414A52F8232004
:10CA7000404B7A601B78002B3EF491AF3E4B1A601E
:10CA8000394B2AB91A6842F008021A60FEF787BFCC
:10CA90001A6822F008021A60FEF781BFFF2A7FF4AD
:10CAA00073A9334E3BB300254FF003080C27607881
:10CAB00018FB00510138784300F5C36000EB850096
:10CAC000042206EB81010135FCF728FC032DEED191
:10CAD000FEF765BF61197819042231440435FCF76B
:10CAE0001DFC0C2DF6D10C34FC2C3EF458AF002567
:10CAF00004F20C67EEE70C24F9E77678142E3FF683
:10CB0000ECACA77838063BD5194FDFF870800025CC
:10CB1000A3782B41D9070DD56901667841F0020150
:10CB200001F0E2010020FDF721F806EB46062E4455
:10CB300047F8260098F81A3083B1637873B103215F
:10CB400011FB03510C20013B584300F5C360042244
:10CB500007EB810100EB8500FCF74DFB0135032D50
:10CB6000D6D1FEF71CBF00BFECCEFF1FBCC6FF1F17
:10CB7000F0CEFF1FFBCFFF1FECCFFF1F0CC0FF1F2E
:10CB8000022F3FF601A9790141F0020101F0E20113
:10CB90000020FCF7EBFFAB4BAB4D9B7E06EB460654
:10CBA0003E4445F82600002B3EF4F9AE6278002A98
:10CBB0003EF4F5AEA078032111FB02010C23013AEB
:10CBC000534303F5C363042205EB810102FB0030EC
:10CBD000FCF711FBFEF7E3BE72789C4B0A2A0CD8D7
:10CBE000DFE802F006151A1F252D32373C414500BB
:10CBF00097491A6809680A441A601A68954B002A0E
:10CC00003AD11A6842F008021A60FEF7C8BE90498D
:10CC10001A680968521AEFE78D4A196812684A4380
:10CC2000EAE78B491A68096892FBF1F2E4E7884A5F
:10CC30001868116890FBF1F201FB1202DCE78449ED
:10CC40001A6809680A40D7E781491A6809680A43DF
:10CC5000D2E77F491A6809684A40CDE77C490A68EB
:10CC6000D2430A60C9E71968794A1160C5E7784A72
:10CC7000196810681860F8E71A6822F008021A604C
:10CC8000FEF78DBE714B1B68C6F80330FDF75CFCE8
:10CC9000FEF785BE7378052B3EF681AEDFE803F024
:10CCA000030A11181F266B4A136803F00F03136061
:10CCB000FEF775BE674A136823F010031360FEF792
:10CCC0006EBE644A136823F020031360FEF767BE4C
:10CCD000604A136823F040031360FEF760BE5D4AAC
:10CCE000136823F080031360FEF759BE594A136896
:10CCF00023F480731360FEF752BE71782E293FF63D
:10CD0000ECAB554A02EB81021365FEF748BE524B6D
:10CD10004E4AD3F80C1111604D4AD3F8101111602E
:10CD2000D3F81421DA614B4AD3F818111160D3F803
:10CD30001C2183F84520D3F82021DA64D3F824217C
:10CD40009A6493F82811454A505C08B10120505468
:10CD5000002283F82C21FEF722BE00F085FEFEF7AC
:10CD60001EBE00F082FEFEF71ABE00F07FFEFEF748
:10CD700016BE00F07DFEFEF712BE00F07AFEFEF752
:10CD80000EBE00F077FEFEF70ABE334B00221A7685
:10CD9000FEF705BE72782AB1012A08D003233B7042
:10CDA000FEF7FDBD2C4B01221A76FEF7F8BD40F2CE
:10CDB000FE718B423EF6E8AF27490A76CB61FEF75B
:10CDC000EEBD254A2548002382F8443082F82C31F4
:10CDD00002F150044FF0FF35194644F82350C15476
:10CDE00001332F2BF9D1194B11761960184BD161F2
:10CDF0001960184B116282F845101960FEF7CFBD1B
:10CE0000127D92070BD440F2FE7293423EF6BCAF05
:10CE1000114A04211176C2F83031FEF7C0BD082353
:10CE20003B70FEF7BCBD0C4B00221A76FEF7B7BD77
:10CE30002B460022E2540133082BFBD123782372C6
:10CE4000FEF7ADBD0CC0FF1FF0CEFF1FECCFFF1FE4
:10CE500008D0FF1FECCEFF1FBCC6FF1F82CEFF1FF6
:10CE60007378012B19D005D3022B1FD003233B70FD
:10CE7000FEF795BD994B01221A70994B994A9B7800
:10CE80001370994B196800230139013311F8010F10
:10CE9000D054082BF9D1FEF782BD0422FA717B71C0
:10CEA00056220823BA713B71FEF779BD8B4B8F4830
:10CEB00001221A708A4B8B4A9B781370002301332E
:10CEC0001918082B11F8091CD154F8D1FEF767BDC9
:10CED0007378032B3EF663ADDFE803F0020F1B20EF
:10CEE000834B1A7EFA7193F84520D3F83031BA712A
:10CEF0001A0A7A713B71FEF752BD7D4B1A7EFA71A8
:10CF000093F84520DB69BA711A0A7A713B71FEF712
:10CF100046BD784B1B687B60FEF741BD764B1B68B6
:10CF20007B60FEF73CBD7278002A7EF438ADB178A4
:10CF300000297EF434AD40F2D24293427EF42FAD0C
:10CF400040F2FF70FCF7F8F8FCF75DF80120FBF702
:10CF5000BDFCFEF724BD0122FEF7B9BC74782CB1EC
:10CF6000012C14D003233B70FEF719BD04220DEBF6
:10CF7000020140F2FB70FCF7D1F9019BD6F80320C7
:10CF80009A4206BF01237B607C60FEF708BDB37840
:10CF90002A2B07D10422594940F2FB70FCF72BF9E8
:10CFA000FEF7FDBC03233B70FEF7F9BC504CD4F8F0
:10CFB0003801002104F59E7281423EF4F0AC52F833
:10CFC00021509D4201F1010520D102EB8503043B74
:10CFD0000138814214D3C4F83801FEF7E0BC444A5A
:10CFE000D2F8381109299DBF481CC2F8380102EB5C
:10CFF0008102092394BFC2F83C313B70FEF7CFBCDD
:10D0000053F8042F43F8042C0131E2E72946D3E713
:10D01000374A0023C2F83831194602F59E7242F8A9
:10D02000231001330A2BFAD1FEF7B9BC0A237B6027
:10D03000FEF7B5BC03233B70FEF7B1BC7378812BC0
:10D040007EF4A2AEB378922B7EF49EAEB379A32B7E
:10D050007EF49AAE7379B42B7EF496AE3379C52BF9
:10D060007EF492AEF378D62B7EF48EAEFBF7F5FE0F
:10D07000FBF750FB0446FBF74DFB001B0028B8BF35
:10D080004042B0F57A7FF6DBFBF71EFC1C4B00221A
:10D090001A604FF0FF32C3F87021C3F87022C3F852
:10D0A0007421C3F87422C3F87821C3F87822C3F836
:10D0B0007C21C3F87C22134B134A1A600120FBF732
:10D0C00005FCFEF76CBC40F2D24293427EF467ACA2
:10D0D000074B012283F86421FEF761BCF0CFFF1FEC
:10D0E0000CC0FF1FF1CFFF1F08C0FF1F0080000012
:10D0F000BCC6FF1FECCFFF1F08D0FF1FE7CEFF1FEE
:10D1000010E000E000C0FF1F78563412364B2DE9C6
:10D11000F04700241C60354B354D1C60354BDFF863
:10D12000E880354FEC611C6085F845406601F6B239
:10D1300046F006010020FCF719FD46F00C0148F806
:10D1400024000020FCF712FD47F824000134032CD2
:10D15000ECD12A4BD97AC1F10801C9B20020FCF701
:10D1600081FF274A00231946904642F823100133D5
:10D17000B3F5807FF9D1234CA37E03BBE37E13B3C9
:10D1800094F824100020FCF745FB637D4BB3FBF7BC
:10D1900029FE30B301232B76BDE8F087B91909EBDE
:10D1A0000700042251440437FCF7B8F80C2FF5D1DE
:10D1B0000C36FC2EE2D0002706F20C69EEE70C26B6
:10D1C000DFF848A0F7E74FF4A766A6F5A761304659
:10D1D000042241440436FCF7A1F8B6F5C36FF4D13C
:10D1E000CEE70023D7E700BFECCFFF1F08D0FF1F1B
:10D1F000BCC6FF1FECCEFF1F0CD0FF1FC0CDFF1F12
:10D2000018D0FF1F0CC0FF1F18D4FF1FF0CEFF1F48
:10D21000F7B50F4C07460E4694E803008DE803006F
:10D220000C49C1F803300C4B8A7000220F704E700D
:10D230001A70FEF7D3F9094A217882F865119DE842
:10D240000300636884E80300184603B0F0BD00BF24
:10D2500000D0FF1FE4CEFF1FFBCFFF1FBCC6FF1F88
:10D26000F7B504461F4A63781370A3785370E378C8
:10D2700093702379937163795371A3791A4D137164
:10D28000E379D3700E4695E80300184B00221A701C
:10D290008DE80300FEF7A2F9154B1A786F462B466E
:10D2A0009AB9327072702A78B2706A78F270EA793C
:10D2B0003271AA7972716A79B2712A79F27197E83A
:10D2C000030083E8030003B0F0BD012AF7D1094849
:10D2D000721EF11D10F8014F02F8014F8A42F9D178
:10D2E000EDE700BFE4CEFF1F00D0FF1FFBCFFF1F05
:10D2F000F0CFFF1FF1CFFF1F014B93F8650170477F
:10D30000BCC6FF1F2DE9F043994B9A4C1B788FB098
:10D310006BB1994B1B78063BDBB2192B04D8974AAB
:10D3200022FA03F3D90702D4002384F8343194F8A5
:10D330003431934E5A1E012A51D89249012BCA68A2
:10D34000079214BF082307238DF81830327894F819
:10D3500066318DF8193000238DF81A30002A33D148
:10D360008B688DF82030884B8DF8272019788DF840
:10D37000211059788DF82210D9798DF823109979D8
:10D380008DF8241059791B798DF825108DF82630E9
:10D3900006A801F0C1FA002800F016837B4B1A782A
:10D3A0009846002A00F01E81794B7A4F1B78013B8A
:10D3B000062B00F21381DFE813F0F100F1005701B2
:10D3C0001101110111017E01012AE1D172480133DD
:10D3D00006AA1A44195CD171082BF8D1D8E7032B9F
:10D3E0003DD1337883BBDFF89C81674F98F802000A
:10D3F00098F801503B7805441D447B781D44FB7927
:10D400001D44BB791D447B791D443B791D44FBF7CA
:10D41000BBF998F80100FBF7B7F93878FBF7B4F9D6
:10D420007878FBF7B1F9F879FBF7AEF9B879FBF743
:10D43000ABF97879FBF7A8F93879EDB2FBF7A4F9E5
:10D440002846FBF7A1F9A9E7012BA7D1524F0025E8
:10D45000785D0135FBF798F9092DF9D19EE7042B8A
:10D460002BD1484FDFF82081B8787D780023012246
:10D470000544154488F8013088F80020C8F80430C5
:10D48000FBF782F97878FBF77FF998F80000FBF753
:10D490007BF998F80100FBF777F998F80700FBF79C
:10D4A00073F998F80600FBF76FF998F80500FBF799
:10D4B0006BF9EDB298F80400C0E7072B37D1337849
:10D4C00053BB304B9F7893F801802F4B8DF8007041
:10D4D0001D785878D9798DF8025047443D449A799F
:10D4E0008DF80300284493F805C08DF8041001441A
:10D4F00093F804E08DF805200A440CEB0203734412
:10D500008DF801808DF806C08DF807E08DF80830A1
:10D510006846FBF79FFC41E7012BF9D11E49002328
:10D520005A5C0DF803200133092BF9D1F0E7082BE1
:10D530007FF434AF144A1349002301205370107054
:10D5400053608A7849788DF800200A4402448DF8A7
:10D5500001108DF802008DF803308DF804308DF83D
:10D5600005308DF806308DF807308DF80820CFE7AC
:10D57000FACFFF1FBCC6FF1FE4CEFF1F110200023F
:10D58000F0CFFF1F0CC0FF1F00D0FF1FB1CEFF1F49
:10D5900078CEFF1F52CDFF1FF1CFFF1FAA4A397867
:10D5A00093688DF8303080238DF831308A238DF8E0
:10D5B000323000238DF833308DF834308DF835302B
:10D5C0008DF836108DF8293007218DF82A300AA8F9
:10D5D000D3688DF828100B9301F09EF900233B705F
:10D5E00088F80030002384F83431337094F86431C3
:10D5F00013B10120FBF76AF906A801F019F90646F4
:10D60000002800F03981914B9DF820201A709DF878
:10D6100021205A709DF822209A709DF823209A713B
:10D620009DF824205A719DF825201A719DF8262016
:10D63000DA709DF8193084F86631FBF76BF8844B8B
:10D640001860844B00221A709DF81830072B0CBF0D
:10D650000123022384F83431237E5A1E012A4AD939
:10D66000052B48D0012247E0DFF8DC913B7899F8A0
:10D67000020099F8015005440A351D44FBF784F86F
:10D6800099F80100FBF780F88020FBF77DF88A20ED
:10D69000FBF77AF80020FBF777F80020FBF774F827
:10D6A0000020FBF771F8EDB23878FBF76DF82846EB
:10D6B000FBF76AF892E7644A507893788DF80C305B
:10D6C0003A788DF80D00802103448DF80E100A334E
:10D6D0008A218DF80F101344002103A88DF8101033
:10D6E0008DF811108DF812108DF813208DF814306C
:10D6F000FBF7B0FB72E70022574B1A70237E042B16
:10D7000004D1524B19780A0640F1618194F8342112
:10D71000082A04D840F25113D340DF0701D4FDF7A3
:10D720005DFF94F83431092B6DD1FAF7F3FFE3680C
:10D730004A4DC01A00282A68B8BF4042904208D912
:10D74000474B1A78012A04BF02221A70FAF7E2FF47
:10D75000E060FAF7DFFF23696A68C01A0028B8BFE3
:10D760004042904208D93E4B5A78012A04BF022217
:10D770005A70FAF7CFFF2061FAF7CCFF6369AA6805
:10D78000C01A0028B8BF4042904208D9344B9A785A
:10D79000012A04BF02229A70FAF7BCFF606194F874
:10D7A000443083B394F82C316BBB2D4A2D481D4671
:10D7B000D15C022940F0FF8050F823104E1C00F08D
:10D7C000F980294A84F828311268C4F80C21274AC4
:10D7D0001268C4F81021E269C4F81421244AE161F6
:10D7E0001268C4F8182194F84520C4F81C210023BD
:10D7F000E26CC4F8202184F84530A26CC4F82421DE
:10D80000012384F82C3194F83431092B04D1227E81
:10D81000022A04BF05222276D4F83821002A00F01B
:10D82000D380092B40F0D080237E012B40F0CC80A8
:10D83000E1691048002350F823508D4240F0C08029
:10D8400005232376C0E000BF0CC0FF1FE4CEFF1FFE
:10D8500068CEFF1F18CDFF1FFBCFFF1F30CEFF1F6D
:10D8600082CEFF1F0CC7FF1FECCFFF1F08D0FF1F8A
:10D87000ECCEFF1FF8C7FF1F03A8FAF79DFF054670
:10D8800000284ED0FAF7B0FF08B184F8676194F829
:10D8900067219DF80C10531CDBB22244092B84F83D
:10D8A000673182F868117FF429AF5E4A94F86811F5
:10D8B00052780023914284F867317FF41FAF5A49B0
:10D8C0005A5C01331644082BF6B2F9D194F8703142
:10D8D000B34222D1554B94F869211A7094F86A2109
:10D8E0005A7094F86B219A7094F86C219A7194F89C
:10D8F0006D215A7194F86E211A7194F86F21DA70C3
:10D90000FAF708FF4A4B4B4A1860002313700322B2
:10D9100084F8342184F867319EE6042384F8343196
:10D92000ECE60AAE3046FBF782FA48B32B46F25CCF
:10D9300001331544082BEDB2F9D19DF83020AA42ED
:10D94000ECD13A4B9DF829201A709DF82A205A7084
:10D950009DF82B209A709DF82C209A719DF82D200F
:10D960005A719DF82E201A719DF82F20DA70FAF75F
:10D97000D1FE2F4B18602F4B00221A70072369E647
:10D98000237E013B012B3FF6B9AEE26940F2FE7304
:10D990009A420CD8FBF726FA48B1E0692349431CA8
:10D9A000E361FBF7EFFA092384F834315AE60023E8
:10D9B0002376A3E6D55401332F2B7FF4F9AE22E76B
:10D9C00001339A427FF437AF0FB0BDE8F08394F88B
:10D9D0003401082804D840F25112C240D207F3D4CF
:10D9E000154DD3F80330D4F830016B6040F2FE736C
:10D9F0009842697012D80D49FBF7D4FB0B49D4F853
:10DA00003001FBF741FB38B1D4F830310133C4F8B1
:10DA1000303165232B70D7E70723FBE707232B70F3
:10DA200000230EE70CC0FF1F24C8FF1FE4CEFF1F1A
:10DA300070CEFF1F77CEFF1F00D0FF1F704710B5BD
:10DA4000074CFAF767FE2368C01AB0F5FA7F05D9CC
:10DA5000044B2022DA60FAF75DFE206010BD00BFA3
:10DA600024D4FF1F00F00F40704770477047704785
:10DA700070477047704770472DE9F04F9E4C2378F0
:10DA800085B033B96FF000436360A360E3600123A6
:10DA90002370257CDFF8A0824DB9E8B2FBF74FF880
:10DAA00008F805000135082DF7D101232374DFF8AC
:10DAB0008CA2924F272500264FF00209F0B2FBF707
:10DAC0003EF818F80630834216D0B31D08F8060059
:10DAD0005AF82330022B0AD0032B02D0012B0BD192
:10DAE00050B17B5D012B08BF07F8059004E018B921
:10DAF0007A5D012A00D17B550136082E05F101051A
:10DB0000DCD17F4DEB69C3B17E4E3778AFB9FAF700
:10DB100001FE7D4B1B68C01A0028EB69B8BF40426C
:10DB200098420AD93846FBF76BFF0120FBF768FFE4
:10DB30000220FBF765FF012333702B6AC3B1734EDC
:10DB40003778AFB9FAF7E6FD714B1B68C01A0028A9
:10DB50002B6AB8BF404298420AD93846FBF750FFBB
:10DB60000120FBF74DFF0220FBF74AFF0123337032
:10DB7000684D2B7B002B40F01682FAF7CBFDE36952
:10DB8000C01A0028B8BF40420A2804DC624B1B6957
:10DB9000DB0700F1E18194F82000002840F00281C9
:10DBA0000A21FBF7DBFD074694F820005B4EFCF7EB
:10DBB00067F8002F40D194F82010490141F0080186
:10DBC00001F0E8013846FBF7C9FDA8BBFAF7A2FD52
:10DBD00094F8202004EB820305EB42115B68B1F856
:10DBE0001CE0C01A00284FF00A03B8BF404203FBF4
:10DBF0000EF3984208DD897A1046FAF775FE94F81C
:10DC000020300121464AD15494F8200087EAE77871
:10DC100056F83030A8EBE77898452BD2FCF722FB7A
:10DC200094F8203006EBC306727982422BD1002192
:10DC30001846FCF7E5FA26E094F8200087EAE77238
:10DC400056F83030A2EBE7729A4235BF06EBC003BC
:10DC500005EB40131979597AFAF746FE94F82080BB
:10DC6000FAF758FD04EB880894F82030C8F804004F
:10DC70000021C7E7FCF7F6FA94F8203006EBC3065C
:10DC800071798842D4D194F82000264B0344019343
:10DC9000254B03440093254B002203EB80031146E0
:10DCA000FCF7B2FB94F8200005EB40139B69BBB175
:10DCB000FBF764F8A0B194F8200005EB40139B69D2
:10DCC00098450DD9FBF79CFE94F82030184A0121A5
:10DCD000D1540F33094AD15C012904BF0221D15428
:10DCE00077B394F82060134B9B5DABBBFAF712FD42
:10DCF00004EB8606706255E030C8FF1F82CEFF1F1E
:10DD00000CC0FF1F77CEFF1F70CEFF1F18CDFF1F67
:10DD100068CEFF1FC0CDFF1FC0F00F4034CDFF1FE6
:10DD200079CEFF1FBBCDFF1F30CDFF1F54CDFF1F8E
:10DD3000B8CDFF1F7CCEFF1F41C8FF1F30CEFF1F95
:10DD400094F82010490141F0080101F0E80138463B
:10DD5000FBF704FD0028C4D194F8203005EB4312F2
:10DD6000D28912B9B94AD35CE3B1FAF7D3FC94F87B
:10DD7000202004EB820305EB42155B6AE989C01A97
:10DD800000284FF00A03B8BF40424B43984209DDD8
:10DD9000AF4DAB5C33B91046FCF7A2FB94F82030D2
:10DDA0000122EA540020FBF7BCFC94F83030DFF885
:10DDB000C8A28DF8080003F0F803C70748BF43F076
:10DDC000010384F83030460742BF94F8303043F006
:10DDD000020384F83030C50648BF94F830309AF812
:10DDE000000044BF43F0040384F83030994B94F8AA
:10DDF000305093F800E0984B1F78984B93F80090C0
:10DE0000974B1E78002319469C4698461A4646FAB8
:10DE100002FB1BF0010F40F0A7800132032AF6D16C
:10DE2000B8F1000F01D08AF80000BCF1000F02D059
:10DE3000884A82F800E009B1874A17700BB1884B15
:10DE40001E70E80709D594F83130D90705D4854B01
:10DE5000DA78012A04BF0222DA70AA0709D594F8F9
:10DE600031309B0705D47F4B1A79012A04BF022267
:10DE70001A716F0709D594F831305E0705D4794BD4
:10DE80005A79012A04BF02225A7104AA94F8201078
:10DE900084F831500323B1FBF3F3134413F9083C26
:10DEA000002B49DA490141F0160103AA01F0F601FD
:10DEB0000020FBF73CFC9DF80E3058060AD594F87C
:10DEC000202002201B2110FB021266498D5C012DCF
:10DED00008BF885419060AD594F8202061490E32EB
:10DEE00011F81200012804BF022001F81200DA061E
:10DEF0000AD594F8202002201B2110FB0212594958
:10DF00008D5C012D08BF88549B060AD594F82030FB
:10DF1000544A0E3312F81310012904BF022102F8EB
:10DF2000131094F82010490141F0160103AA01F0E2
:10DF3000F6010020FBF736FB94F8200000F0B8F85B
:10DF400094F820300133DBB2032B88BF002384F820
:10DF50002030FAF7DFFBE06105B0BDE8F08F01216A
:10DF60000F468C46884658E745FA02FB1BF0010F26
:10DF70003FF453AF40FA02FB1BF0010F7FF44DAFAB
:10DF80000121914049B2084341EA0E0EC0B25FFA46
:10DF90008EFEB9F1000FE2D101234E4619461F460D
:10DFA0009C46984639E700222F4E304B84F82020BB
:10DFB00010460196009311462D4BFCF725FA94F874
:10DFC000200033562B4E002B04EB000393F8323025
:10DFD0001CDB022B01D1335C83B105EB4015697A60
:10DFE000FAF782FC94F82000FCF784FA94F82030C9
:10DFF000E218022182F832100022F25494F82050E4
:10E00000FAF788FB04EB85046060A5E7012B35D1A6
:10E0100094F82030F35C002B9ED094F8200005EBA0
:10E020004013997AFAF760FC94F8200005EB40154C
:10E03000AB7ABBBBFCF754FA94F820301C440122A5
:10E0400084F832200022F25486E700BF7CCEFF1F06
:10E050007FCEFF1F52CDFF1FB1CEFF1F28CDFF1F68
:10E0600053CDFF1F82CEFF1FBBCDFF1F30CDFF1F43
:10E0700054CDFF1F74CEFF1F29CDFF1FFAF74AFBB7
:10E0800094F8202004EB820305EB42125B68928B2C
:10E09000C01A00284FF00A03B8BF404253439842C9
:10E0A000B6DDBAE7335C002BC6D0FCF723FAC3E732
:10E0B0002DE9F04F47017DB285B045F07C01044663
:10E0C00003AA01F0FC010020FBF731FB4FEA440AF0
:10E0D0009DF90E304FF0020B012202FA0AF20BFA00
:10E0E0000AFB03EA0B0B1340DBB20193CD4BDA19A9
:10E0F0005FFA8BFB127A12F0800F02F07F084FF06C
:10E100000000994613D0FAF71AFDB0FA80F35B09C4
:10E1100008F1FF32072A00F2E581DFE812F00E0075
:10E120000E000E000E004201420142014201FAF7C8
:10E1300006FD031C18BF0123EAE7BB4E335D0F2B1E
:10E1400000F2D081DFE813F0CE01100077013C002F
:10E15000A4014D00560066007B00B200E900EF000C
:10E16000CE0112011C015C0245F0140103AA01F06A
:10E17000F4010020FBF7DBFA45F0060106EB84070B
:10E18000CDB29DF80D307B6029460020FBF7E6FA02
:10E190000222386121460020FBF7F6FA40F2FF72B6
:10E1A00029460020FBF723FAA8F1020803222146A2
:10E1B0000020FBF70CFBB8F1010F0FD802230EE093
:10E1C000019B002B00F08E8145F0020101F0E2017D
:10E1D0000020FBF7CBFC954B43F824000423335578
:10E1E00080E1BBF1000F00F07D812046FBF708FCC9
:10E1F0000623F4E70322214600204F44FBF7E7FA09
:10E2000045F008017A6801F0E8010020FBF7EFF91A
:10E210000723E4E7BBF1000F40F0648145F00801FB
:10E22000CDB24F445A4629465846FBF7E0F97A6882
:10E23000294652425846FBF7DAF90823CFE7BBF1EB
:10E24000000F00F04F8145F0020101F0E2010020D3
:10E25000FBF78CFC002245F00801804601F0E80144
:10E260001046FBF7C4F9714A52F82430A3EB0803B7
:10E2700042F82430214603220020B944FBF7A7FAD4
:10E2800045F00601D9F8042001F0E6010020FBF773
:10E29000AEF9424607F0E0010020FBF7BAF9002290
:10E2A00021461046FBF770FA092398E70020FBF798
:10E2B00038FA40FA0AF0C10740F1148145F0080A23
:10E2C00000225FFA8AFA10465146FBF790F90222C3
:10E2D00021460020FBF758FA002245F002011046C3
:10E2E00001F0E201FBF795F9002207F0E00110468A
:10E2F000A8F10308FBF78DF9B8F1010F3ED84F44A0
:10E30000022221460020FBF73FFA7A68514652422A
:10E310000020FBF76CF90A2361E7BBF1000F00F066
:10E32000E1800B235BE7BBF1000F40F0DB8045F0A1
:10E33000020101F0E2015846FBF718FC45F0080124
:10E3400080465A4601F0E8015846FBF750F9022290
:10E3500007F0E00198FBF2F25846FBF75AF95A46EB
:10E3600021461046FBF710FA0D2338E70020FBF793
:10E37000D8F940FA0AF0C20740F1B4800E232EE724
:10E3800006EB840745F006013A6901F0E60100203A
:10E39000FBF72DF93A7921460020FBF718FA002304
:10E3A0001DE7214E325D0F2A00F29C80DFE812F05B
:10E3B0009A00100040005E006D008C009A009D00E5
:10E3C0009A009A00CE00DB00B60003013601280156
:10E3D00045F0140103AA01F0F4010020FBF7A7F9AE
:10E3E00006EB84039DF80D205A602146022200208E
:10E3F000FBF7CAF945F0060140F2FF7201F0E601B1
:10E400000020FBF7F4F8032221460020FBF7DFF998
:10E41000B8F1060F3FF4D2AEB8F1080F7FF4DEAECC
:10E42000CCE600BFC0CDFF1F68C8FF1F1CCDFF1F7B
:10E43000B8F1060F15D106EB84035A6802F0040206
:10E4400042F0010221460020FBF7C1F945F0080126
:10E4500059F8072001F0E8010020FBF7C8F8032372
:10E46000BDE6B8F1080FF1D10322EBE7A8F10502F0
:10E47000012A07D8019A2AB1B8F1060F3FF4AEAECF
:10E480000F23ACE673B30C23A9E6B8F1050F16D140
:10E4900006EB84035A6802F0040242F002022146AD
:10E4A0000020FBF794F959F8072045F00801524283
:10E4B00001F0E8010020FBF79AF805238FE6B8F198
:10E4C000070FF0D10322EAE7A8F10502012A06D8D6
:10E4D000BBF1000F03D0B8F1050FD1D16EE6002BD0
:10E4E0007FF496AE05B0BDE8F08F002BFAD1A8F10D
:10E4F0000708B8F1010F0AD906EB840221465268D9
:10E5000002F0040242F001021846FBF760F94F44A2
:10E5100045F008017A6801F0E801F9E6002BE1D145
:10E52000A8F10708B8F1010F0AD906EB84022146C9
:10E53000526802F0040242F002021846FBF747F963
:10E540004F4445F008017A685242E4E7002BC9D0F5
:10E5500045F0020101F0E2010020FBF707FB06EBAA
:10E560008403D861DDE6002BBCD145F0020101F047
:10E57000E20118460193FBF7F9FAB944019B89F8C7
:10E580000D3045F006018046D9F80420184601F008
:10E59000E601FBF73EF806EB8402019BD2691846C0
:10E5A000904407F0E001022298FBF2F2FBF731F809
:10E5B000019B1A46D4E60020FBF7B3F840FA0AF0B4
:10E5C000C3078FD5002245F008010E23104601F045
:10E5D000E8013355FBF70BF8214602220020FBF738
:10E5E000D3F8002245F00201104601F0E201FBF7EA
:10E5F00010F8002207F0E0011046FBF70AF871E777
:10E60000214602220020FBF7BFF845F00801002256
:10E6100001F0E8011046FAF7EAFFAFE606EB8403E3
:10E620001A79B8E6024B1A5C0AB901221A547047EB
:10E6300068C8FF1F024B1A5C0AB10F221A547047B8
:10E6400068C8FF1F014B185C704700BF68C8FF1FF8
:10E650000E4B1A6802F01F02052A0AD0062A0ED0B5
:10E66000042A10D11A690A4992B20A8045221A6016
:10E6700070471A69064992B28A804622F7E71A69FA
:10E68000034992B24A804422F1E700BF00B00B4038
:10E6900090C8FF1F0E4B41F230013A205A5842F009
:10E6A00000625A5041F23C015A5842F000625A50FE
:10E6B00003F5E8230C229A6006491022DA60002252
:10E6C0005A620A624A628A6244221A6000F07ABA86
:10E6D0000070044000B0044009282BD8DFE800F0A7
:10E6E000050A0D1014172A2A1A25134B1888C0F38F
:10E6F0000B107047104B5888F9E70F4B9888F6E7D6
:10E700000D4B188880B270470B4B5888FAE70A4BBC
:10E710009888F7E7084B588883B24FF498705843AD
:10E720004FF6FF7390FBF3F07047034B988883B26A
:10E730003420F4E70020704790C8FF1F30B52E4DFD
:10E7400041F23C042B5943F010032B512B4B4FF457
:10E7500000749C646FF4F875DC64A3F51833A4F1BD
:10E760003E542C441C604FF400545C60244C1C60EC
:10E770001C68E401FCD50138072834D8DFE800F034
:10E78000312F2D2B293327041E4858601E4B0020A3
:10E7900058631E4818601E484FF0806400EA8145A7
:10E7A000C3F88040C3F88450FAB100EA8240C3F84D
:10E7B0009040C3F894004FF08460C3F8A000C3F801
:10E7C000A410AAB1C3F8B000C3F8B42030BD1148FA
:10E7D000DBE71148D9E71148D7E71148D5E71148D9
:10E7E000D3E71148D1E71148CFE7C3F89020E2E71B
:10E7F000C3F8B02030BD00BF0070044000A004404A
:10E800000F0080508320FC01004002400F00800078
:10E810000000FC1F8720FE028720FE0B8720FE0ED3
:10E820008720FE1D8720FE4A8720FE958720FE0553
:10E83000384AD2F88030C3F30363022B5FD0D2F89A
:10E840009030C3F30363022B5BD0D2F8A030C3F344
:10E850000363022B06D0D2F8B030C3F30363022B5C
:10E8600056D103231B0103F1402202F50032D2F8F6
:10E870008010C1F303410170D2F8801011F48011AF
:10E8800018BF01218170D2F8801011F4001118BF57
:10E89000012141704178B1BBD2F88410C1F38A41A3
:10E8A00003F1402303F500334160D3F88810090ECB
:10E8B0000172D3F88810090C4172D3F88810090A44
:10E8C0008172D3F88810C172D3F88C10090E0173CD
:10E8D000D3F88C10090C4173D3F88C10090A81739A
:10E8E000D3F88C30C373D2F880309B024CBF4FF00A
:10E8F00084634FF08063C2F88030012070470023AA
:10E90000B0E70123AEE7D2F8841021F06041C7E7F9
:10E910000020704700400240184AD2F87031C3F31B
:10E9200003630C2B10B527D04478436804B3C3F3BA
:10E930001103C2F874318368104A1BBAC2F87831E7
:10E94000C3681BBAC2F87C318378002C14BF4FF027
:10E9500042624FF040620BB142F4801203781B0414
:10E9600003F470231343054A0120C2F8703110BD2F
:10E97000034901EA8343DCE7002010BD0040024068
:10E980000000FC1F0B4B4FF00062C3F870214FF4E6
:10E990008022C3F87421084AC3F878216FF4847187
:10E9A000A2F166320A44C3F87C21044AC3F87021FC
:10E9B000704700BF00400240785634120000080C37
:10E9C00010F0040F0A4B10D04FF48042C3F8A0207F
:10E9D000C2064CBF074A084A9A6310F00800074B6A
:10E9E0001ABF01221A70187070474FF48072F3E753
:10E9F0000090044000010A000001090028D4FF1F14
:10EA000038B50446F9F760FF0C49E517C1E9004540
:10EA1000D1E900452B0243EA14632202C1E9002335
:10EA2000074A00231360074A1360074AD364536000
:10EA3000D364BDE83840F9F743BF00BF68CDFF1F7E
:10EA40002CCDFF1F20CEFF1F009003400D490E4A22
:10EA50004FF4804330B5C1F8A0300C4B00240025A2
:10EA6000C3E9004500231360094A1360094AD364CF
:10EA70005360D364084B1B7813B94FF480738B63D6
:10EA800030BD00BF0090044020CEFF1F68CDFF1FA7
:10EA90002CCDFF1F0090034028D4FF1F10B9024B5C
:10EAA00009011960704700BF64CDFF1F08B908460F
:10EAB00086E7704730B9044BD3E90023100A40EAD7
:10EAC000036070470020704768CDFF1F08B90846F3
:10EAD00096E770472A4941F23C0210B58B58294C01
:10EAE00043F000738B50284B5A6D42F004025A6574
:10EAF0001A6822F018021A605A6D22F001025A6553
:10EB0000D3F8842042F0C002C3F8842000214FF6DD
:10EB1000FF72D96459609A60D3F8802042F00102F4
:10EB2000C3F88020D3F8802042F02002C3F8802070
:10EB3000D3F8802042F01002C3F880205A6D42F0D2
:10EB400001025A651A6842F008021A604FF4E06345
:10EB5000236363630D4B0E4A186943091B0100F0E0
:10EB60001F001360FFF72CFF0846FFF749FF4FF423
:10EB70008043C4F8A0305720BDE8104000F022B810
:10EB8000007004400090044000900340C0CDFF1F7F
:10EB900064CDFF1FFEE74FF0E023084AC3F8082DBD
:10EBA000074A4CF22053D3814DF62813D3811388A2
:10EBB00023F001031B041B0C13807047008000002E
:10EBC00000200540802800F01F014FF001030F4A8C
:10EBD00004DD8B40C2F88C31D3607047402804DDDF
:10EBE0008B40C2F8883193607047202804DD8B4049
:10EBF000C2F8843153607047404200F01F0058BF94
:10EC000041428B40C2F880311360704700E100E060
:10EC1000802800F01F024FF001030D4903DD9340EF
:10EC2000C1F88C307047402803DD9340C1F888302C
:10EC30007047202803DD9340C1F88430704740427C
:10EC400000F01F0058BF42429340C1F88030704727
:10EC500000E100E0074B1A78D2B2012A02D1222942
:10EC600003D15A7001225A7070472129FAD100222B
:10EC7000F7E700BFA4C8FF1F70B5154611B91B4BBD
:10EC8000197070BD022903D1184B01221A7070BD92
:10EC900004291AD1154B5B78012B25D19488402C7F
:10ECA00028BF402400235E1CDBB2A34207D300230D
:10ECB0001A4602211846BDE8704000F047BF2A6896
:10ECC000D05C00F0C3F83346EDE7032906D1074ACC
:10ECD0005378012B08D100239370E9E7052901BF80
:10ECE000024B00221A705A7070BD00BFA4C8FF1FEB
:10ECF00010B50446204600F0C1F80028FAD110BD36
:10ED0000704738B50A4C012502460B4600202946BB
:10ED1000A57000F0F5FA224618B10023A370122066
:10ED200038BD937803F0FF00002BFAD138BD00BF47
:10ED3000A4C8FF1FF8B506460F4600F0F4FC0E4BC2
:10ED40001A78012A16D15B78012B13D100F000F953
:10ED500088B10025ECB2A74205D821463046BDE86F
:10ED6000F840FFF7CEBF301900F0D6F80135002883
:10ED7000F0D0F2E70C20F8BDA4C8FF1F08B5402171
:10ED80000248FFF7D7FF00F095F808BDA7C8FF1F9E
:10ED900038B5054600F0A8F80B28044609D14021F3
:10EDA0000548FFF7C7FF28B92846BDE8384000F0FE
:10EDB0009BB80024204638BDE7C8FF1F70B50C463D
:10EDC000461E00250CB9284670BD16F8010FFFF746
:10EDD000DFFF013C002818BF0B25A4B2F2E738B5CD
:10EDE000451E002415F8010F08B9204638BDFFF76D
:10EDF000CFFF002818BF0B24F4E707B5012300223A
:10EE000000930649064B104600F020FA002814BF74
:10EE10001B20002003B05DF804FB00BF79EC00006C
:10EE200055EC000038B50C46054600F097F8A042B6
:10EE30000AD32C440020A54207D000B138BD15F8F4
:10EE4000010B00F051F8F6E70B2038BD10B50A4A67
:10EE5000117840290ED05378D4180133DBB2402BFF
:10EE6000A07001F101014FF00000117014BF537048
:10EE7000507010BD0B2010BD27C9FF1F10B50C4AE4
:10EE8000117891B192F84230D4180133DBB2A478F2
:10EE90000470402B4FF0000001F1FF31117014BFDE
:10EEA00082F8423082F8420010BD0A2010BD00BF37
:10EEB00027C9FF1F014B1878704700BF27C9FF1FE4
:10EEC000024B1878C0F14000C0B2704727C9FF1F3D
:10EED000034B00225A7083F842201A70704700BF1B
:10EEE00027C9FF1FFFF7F4BF10B50A4A1178402960
:10EEF0000ED05378D4180133DBB2402BA07001F14F
:10EF000001014FF00000117014BF5370507010BD1C
:10EF10000B2010BD6AC9FF1F10B50C4A117891B1C2
:10EF200092F84230D4180133DBB2A4780470402B3D
:10EF30004FF0000001F1FF31117014BF82F8423030
:10EF400082F8420010BD0A2010BD00BF6AC9FF1F31
:10EF5000014B1878704700BF6AC9FF1F024B187831
:10EF6000C0F14000C0B270476AC9FF1F034B0022C6
:10EF70005A7083F842201A70704700BF6AC9FF1F99
:10EF8000FFF7F4BF70B50546007801F093F90278F9
:10EF90000023D9B2914207D25C1C03EB83030344E4
:10EFA0005E786B789E4227D1174C2B7A342202FB75
:10EFB0000142D67813B334234B43E218907886424B
:10EFC0000CD000F0030204330C2010FB0230211897
:10EFD000205C0B894A68497800F090FBD4F89C309B
:10EFE00083B12A46287812F8081F00290CBF032194
:10EFF0000521BDE8704018472346CAE793780133DE
:10F000009370D8E770BD00BFB0C9FF1F2DE9F04F66
:10F0100085B00D4690468DF80F0001F04BF9022D9A
:10F02000064647D1077800235C1CDBB2BB4210DBED
:10F030004FF00009DFF8B0B0CA465FFA89F4A74282
:10F0400012DC284BD3F89C30002B45D105B0BDE82D
:10F05000F08F03EB830333440DF10F00DA78597816
:10F0600001F0E2F92346DFE704EB84043444E3785B
:10F07000A2886178CDF804A0A07800900DF10F006F
:10F0800001F0B0F9A378032B05D15A4661789DF8B9
:10F090000F0001F031FA6178E37841F0100141EAA4
:10F0A000C3110022C9B20DF10F0001F0EDF909F111
:10F0B0000109C2E7002DC4D10A490378342000FBBE
:10F0C00003138A1C3633294634329A42B9D002F8E7
:10F0D000341C02F8331CF7E7424629469DF80F001E
:10F0E0009847B3E7B0C9FF1F85EF0000F0B40C7874
:10F0F00004F06004202C1D4632D14C78042C1DD025
:10F100000AD8012C04D003D3022C20D0032C12D017
:10F1100000202880F0BC7047212C1BD004D8202C64
:10F12000F6D1F0BC00F040B9222C16D0232CEFD140
:10F13000F0BC00F049B9F0BC00F049B902241C80D1
:10F140001468002525701468671C17606570F0BC92
:10F1500000F056B9F0BC00F01FB9F0BC00F076B971
:10F16000402C06D1044CD4F8A04014B1A446F0BC05
:10F170006047CD20CEE700BFB0C9FF1F73B504467E
:10F18000007801F097F863680093A27A637A43EA03
:10F190000223ADF8043002780023D9B2914207D29D
:10F1A0005D1C03EB830303445E7863789E4225D1A4
:10F1B000174D237A342202FB0152D67803B334234D
:10F1C0004B43EA18907886420CD000F003020433D7
:10F1D0000C2010FB02302918285C0B894A684978FA
:10F1E00000F08CFAD5F89C3033B1227A20785AB1ED
:10F1F00004F108020521984702B070BD2B46CCE708
:10F20000937801339370DAE76A460321F3E700BF8E
:10F21000B0C9FF1F07B543680093437A817A43EA78
:10F220000123ADF80430084BD3F89C3002462BB1D3
:10F23000017A007829B108320521984703B05DF8BA
:10F2400004FB6A460421F8E7B0C9FF1F2DE9F84323
:10F2500005460F461646984601F02CF802789DF8B0
:10F26000203001328146D2B20021284601F09EF8BA
:10F270000446E8B9164A1749284600F086F999F875
:10F280000000154B342200FB022209F101011A444F
:10F2900099463433934201F105010CD14146284689
:10F2A00000F074F8044618B9C9F89C70C9F8A06059
:10F2B0002046BDE8F88311F8050C03F8340C11F86A
:10F2C000040C03F8330C03F8324C03F8314CE0E73C
:10F2D000EDF000000DF00000B0C9FF1F08B5074BAE
:10F2E0000022C3F89C20C3F8A02000F0A1F918B9AF
:10F2F000BDE8084001F06EB808BD00BFB0C9FF1FEF
:10F300002DE9F041984605460E46174600F0D2FF1B
:10F3100004780023D9B2A14207D2013303EB830260
:10F32000024412F8042CB242F4D1174C34234B435C
:10F33000E218D07892F802E0A0EB0E01C9B20429DD
:10F3400002D1C120BDE8F08100F003010130C0B25C
:10F350004FF00C0C0CFB0133D070A0EB0E001C44E2
:10F36000C0B2012825716671A760A4F80C8007D18E
:10F3700043463A4631462846BDE8F04100F0BEB962
:10F380000020BDE8F08100BFB0C9FF1F014B002085
:10F390001960704754CAFF1F024B0979197100F0B8
:10F3A0008DBF00BF54CAFF1F13B5002402AA1C80E2
:10F3B000044B42F8041D0979197100F08DFF02B069
:10F3C00010BD00BF54CAFF1F00201880704730B422
:10F3D0000C460221198021796488084D012C29717D
:10F3E00002D130BC00F08EBF022C02D130BC00F044
:10F3F00095BF0020188030BC704700BF54CAFF1F63
:10F4000030B40C460221198021796488074D012C03
:10F41000297102D130BC00F08DBF022C02D130BC6A
:10F4200000F09ABF0020188030BC704754CAFF1FFC
:10F43000044B054A19795B791171137203210A2370
:10F44000FFF75EBF54CAFF1F4CC0FF1FF8B500276F
:10F450001F808B780B4CA371C3F340035A0063F3F6
:10F46000000206466271FFF7E3FF256845B1A37904
:10F4700013F002021ABF3A46222121213046A84742
:10F480000020F8BD54CAFF1F034B00F108021B689F
:10F4900000780521184700BF5CCAFF1F70B5094DF1
:10F4A00004462A1D012100F0D7FF802201212046B9
:10F4B00000F0EAFF2B68207800220A21BDE87040A6
:10F4C000184700BF5CCAFF1F37B501210DF10702C5
:10F4D000044600F0C1FF9DF80730074D802B04D192
:10F4E0002A790121204600F0CFFF2B6820780022E6
:10F4F0000B21984703B030BD5CCAFF1F436805214C
:10F500005A7800F0C1BF73B50122002405460126D8
:10F51000002100F089FF334621468DE8500010227B
:10F52000284600F05FFF22462146284600F07CFF77
:10F53000234621468DE850001022284600F052FF55
:10F5400031460222284600F09FFF32460621284617
:10F5500000F09AFF22469021284600F095FF044BC8
:10F5600028781B682246214602B0BDE87040184743
:10F570005CCAFF1F42783AB9C178C90141F0100155
:10F5800001F0900100F080BF704773B50C468DF814
:10F59000070001F00DFA1F4D2C600446002836D1FB
:10F5A0001D4A9DF80700102100F0A6FF1B4A0446E3
:10F5B00012219DF8070000F09FFF194A044314210F
:10F5C0009DF8070000F098FFE4B20443154A9DF847
:10F5D0000700132100F090FFE4B20443124A9DF8A3
:10F5E0000700172100F088FF02AEE4B204430F4A7F
:10F5F00016F8010D162100F07FFFE4B20443032248
:10F600000121304600F040FF0323E4B22B71204675
:10F6100002B070BD5CCAFF1F07F50000FDF40000DA
:10F620009DF40000C9F4000075F5000089F40000A5
:10F6300037B502AD174B05F8010D00221021284601
:10F640001A6000F05BFF12210446284600F056FFC6
:10F6500014210443284600F051FFE4B2044313216F
:10F66000284600F04BFFE4B204431721284600F07F
:10F6700045FFE4B204431621284600F03FFFE4B200
:10F68000204310F0FF0003D19DF8070001F09CF922
:10F6900003B030BD5CCAFF1F1FB501218DF8070004
:10F6A0000DF10E020DF1070000F0D6FE0DF10F0274
:10F6B00006210DF1070000F0CFFE9DF80E30802BE3
:10F6C00018D19DF80F309B0714D59DF8070000F066
:10F6D000EFFD012804460DD172B60DF1070000F0D0
:10F6E00029FB002221460DF107008DF80E2000F0C5
:10F6F000CBFE62B69DF80E0004B010BD73B50C468B
:10F7000015461E468DF80700FFF7C6FF802808D073
:10F7100033462A4621460DF1070000F0A7FA02B051
:10F7200070BD0020FBE77047062812D88000012931
:10F73000C0B201D10230C0B2074AC0F34703122160
:10F7400001FB03231A884FF6FF739A4208BFFF207C
:10F750007047FF20704700BF64CAFF1F2DE9F041CA
:10F76000314C324D324E4FF0000884F800814FF496
:10F77000107285F840020F462846FF2102F072F908
:10F780004FF4806241463046C5F8446202F06AF99F
:10F7900094F80C3143F0800384F80C3194F80C3168
:10F7A0001B06FBD4234BFF221A7094F80C3143F054
:10F7B000400384F80C31204B196897B341F00041A5
:10F7C0001960194B310AC6F3074201F0FE0183F8B4
:10F7D0009C1083F8B020320E83F8B420174AC5F885
:10F7E0004822102283F80821012283F89420BF22A6
:10F7F00083F8802093F8002102F07F0283F8002133
:10F8000093F8842042F0010283F8842093F8842046
:10F8100042F0100283F8842084221A770020BDE889
:10F82000F08121F00041CBE70020074064CAFF1FB0
:10F8300000D6FF1F56C0FF1F0070044000D8FF1FF6
:10F840000D4B93F80C2102F0BF0283F80C21BF226C
:10F8500083F8802093F8842002F0FE0283F884204D
:10F8600093F8942002F0FE0283F894201A7F02F0AD
:10F870007B021A770020704700200740F7B5082365
:10F8800004248DE81800B1F803300D788878B3F5BA
:10F89000007F81BF0023CB7002230B71062D71D82E
:10F8A000AB00DCB2012804BF0234E4B24FEA540ECC
:10F8B000354C122707FB0E474FF6FF76B7F800C00E
:10F8C000B4455FD14E78032E5CD801285AD897F8FA
:10F8D0000FC0BCF1FF0F04BF4FF0000C87F80FC042
:10F8E000B1F803C0122101FB0EFE04EB0E0743EA40
:10F8F0004003BA73FA7B7E7402F0010213435BB2D9
:10F90000D4F84822C7F80220D9B2F9733874D4F871
:10F91000447224F80EC01BB207EBC30E81F0010144
:10F92000CEF80420AEF802C04FF0080E07F833E01E
:10F9300007EBC10ECEF80420AEF802C012FA8CF22A
:10F940004FF0480E07F831E0C4F8482228B917F8FC
:10F95000332062F07F0207F8332002AA02EB800016
:10F960002DB20A4950F8082C11F82530012E0CBF91
:10F97000164642F001063343DBB201F82530002081
:10F9800003B0F0BD9520FBE764CAFF1FC02007400D
:10F99000084610B51146FFF7C7FEFF281DD0104BD3
:10F9A0001221C0F3470001FB0030D3F84422C37B8F
:10F9B0001CB283F0010312F8341001F07F0102F849
:10F9C000341012F8331001F07F0102F833104FF0B9
:10F9D000FF338372C372002010BDC42010BD00BF6E
:10F9E00064CAFF1F73B50C468DF807001146204608
:10F9F0001646FFF799FEFF28054620D021463246DD
:10FA00000DF10700FFF7C4FFC5F3470312210D4DA9
:10FA100059436B18D5F848221888121AC5F848229D
:10FA200024B2094A002002F824004FF0FF326A5441
:10FA30009A705A70DA701A715A7102B070BD9620BD
:10FA4000FBE700BF64CAFF1FC02007402DE9F0415B
:10FA50000E468046114630461746FFF765FE0C4DB0
:10FA6000C0F34700122303FB0050C47BFF2C0DD0D2
:10FA70003A4631464046FFF78BFF24B2D5F8442280
:10FA800012F8343063F07B0302F83430BDE8F081C3
:10FA900064CAFF1F10B5084600211446FFF744FE54
:10FAA000084AC0F34700122101FB0020D2F844327B
:10FAB000C27B03EBC2035A68136823605368636018
:10FAC00010BD00BF64CAFF1F10B50C46204611468A
:10FAD000FFF72AFEFF281AD024B2104B13F8243067
:10FAE000DBB213F00C0F12D09B0712D40C4BD3F8DF
:10FAF000443213F83020D2090DD180F00100C0B299
:10FB000013F83030DB0914BF0320002010BD05209E
:10FB100010BD012010BD032010BD00BFC020074054
:10FB200064CAFF1F08B5FFF7FFFD074A1223C0F3A1
:10FB3000470003FB0020C37BFF2B1EBFD2F84422EB
:10FB4000002102F8331008BD64CAFF1F2DE9F041FF
:10FB50000846002190461F46FFF7E6FD2249C0F304
:10FB60004700122404FB0014E57BFF2D39D02288C6
:10FB70004FF6FF7093B2834233D0D1F8441285F030
:10FB8000010011F9300000282BDB2EB287B901EB00
:10FB9000C60338465A80D4F802205A6011F835203E
:10FBA00002F0400262F0770201F83620BDE8F081F1
:10FBB00001EBC602BB424FF0000028BF3B46678105
:10FBC000C4F80680207360735380C2F8048011F873
:10FBD000353003F0400363F0770301F83630BDE8B9
:10FBE000F0819420BDE8F08164CAFF1F2DE9F04147
:10FBF0000C460646114620461546FFF795FD194B63
:10FC0000C0F34700122202FB003090F80FE0BEF173
:10FC1000FF0F24D027B2144A6CB1407C012D0CBFD9
:10FC200014211821012818BF41F0010112F8270002
:10FC3000014302F8271012F827106FF3410102F870
:10FC40002710D3F84432002203F83E203DB92B465A
:10FC50002A4621463046BDE8F041FFF777BFBDE8B0
:10FC6000F08100BF64CAFF1FC02007402DE9F041AA
:10FC70000C462046012117469846FFF755FDFF2800
:10FC800036D01C4BC0F34700122202FB0030D3F8E1
:10FC9000446290F80FE016F93E30002B28DB23B2C7
:10FCA000154A12F8235015F0020521D10188C0F839
:10FCB00006701FFA88F242818A42D8BF11460FFAB5
:10FCC0008EF206EBC2030573457359805F602CB951
:10FCD000C82306F832302046BDE8F08116F83E30E1
:10FCE00003F0400363F0770306F832302C46F2E766
:10FCF0009324F0E764CAFF1FC0200740034B044869
:10FD000083F898100122114600F0BEBB0020074086
:10FD1000A4CCFF1F054B0648002283F894208022C4
:10FD200083F80C210121FF2200F0AEBB0020074028
:10FD3000A4CCFF1F38B51A4C94F8002102F07F02C2
:10FD400084F8002194F80C2102F0DF0284F80C21E1
:10FD500094F8802042F0200284F8802094F88420D7
:10FD600002F0DF0284F8842094F8942002F0DF028D
:10FD700084F8942094F8942042F0040284F89420AB
:10FD800044F62065013DADB200F0BCFE002DF9D176
:10FD900094F8943003F0FB0384F8943038BD00BF2E
:10FDA000002007402DE9F04FD84DD94C95F88070D0
:10FDB00095F8843095F8906087B0FF221F4094F842
:10FDC00040328DF809208DF80C308DF80D2000237D
:10FDD00001210DF1090204F510708DF80E30049325
:10FDE0008DF815308DF816308DF80F308DF81430F1
:10FDF00000F032FB95F80C31D907F6B20FD59DF81B
:10FE00000930802B0BD195F8003103F07F0385F882
:10FE1000003195F80C3103F0DF0385F80C317A07D7
:10FE200011D5BA4B042093F8A41093F8A02083F8BE
:10FE3000800006AB42EA012223F80E2D03A912200E
:10FE4000049300F06DFBFB074BD5B04DB048012388
:10FE5000BF2685F8803085F8886095F894300027B3
:10FE600043F0020385F894304FF4107285F89870CF
:10FE7000FF2185F8007101F0F5FD4FF480623946ED
:10FE8000D4F8440201F0EEFDD4F8443203F50073D7
:10FE9000C4F848329F4BFF221A7095F8943003F053
:10FEA000FD0385F8943095F80C3143F0400385F854
:10FEB0000C319F2385F88C6085F8843095F8943058
:10FEC00003F0DF0385F8943003A9102000F028FB2D
:10FED00095F8943003F0DF0385F8943007B0BDE85F
:10FEE000F08F3D0740F19380884B082283F88020F3
:10FEF0003309C6F3C000062B8DF80D308DF80F00C6
:10FF000000F2F480C6F3800202EB830208B10232F1
:10FF1000D2B2D4F8446206EBC201C2F34705D1F86D
:10FF200004E04988ADF81510122101FB0541CDF818
:10FF300010E091F80FC08CF0010C81F80FC016F89A
:10FF4000321082F0010A5FFA8AFAC1F380110FFAC7
:10FF50008AF881F00101890106EBC80906F838101A
:10FF6000002800F0D980DFF8ACB19BB99BF80020E5
:10FF700082B9FF2219468BF8002003A81A46019384
:10FF8000FFF706FD019B06F838301A46194603A80C
:10FF9000FFF7DCFD9BF80030012B04D09DF80D30FD
:10FFA000002B00F0AD80122101FB0541BDF81500CA
:10FFB0008B894A8903449BB293428B8109D3B1F860
:10FFC00000E0C0B2864540F09380897B012940F073
:10FFD0008F80122101FB0544D4F8061020881944B3
:10FFE000D31A8342D8BF98B2A9F80200C9F8041006
:10FFF00016F83A3003F0400363F0770306F8383020
:020000021000EC
:10000000424A92F8943003F0DF0382F89430B80744
:1000100017D53E4C022384F8803094F8883094F849
:100020008C2003A9134016208DF8143000F078FAC4
:10003000BF2384F8883094F8943003F0DF0384F809
:100040009430F9061CD5314C202384F880301023DD
:1000500084F8803003A9142000F062FA94F80C317F
:1000600043F0200384F80C3194F8003143F080030E
:1000700084F8003194F8843043F0200384F884300D
:10008000BA060DD5214C202384F8803003A9132013
:1000900000F046FA94F8843003F0DF0384F88430EB
:1000A0003B067FF51BAF0DF10A02FF23102103A8C9
:1000B0008DF80D3000F0D0F99DF80A30134C012B6B
:1000C00004BF8DF80F3000224FF0800308BF8DF879
:1000D0000D2003A984F88030172000F021FA94F84D
:1000E000943003F0DF0384F89430F7E6FF2210E742
:1000F000122202FB0544D4F806200492ADF8153014
:1001000003A99DF80D0000F00BFA79E700200740E5
:1001100064CAFF1F56C0FF1F6BB916F832202F4963
:1001200002F03C02342A35D101238DF80E309EF8BE
:100130000030DB090B70122101FB05414FF6FF7304
:100140004A899A42DCD0BDF815E08B8973449BB292
:100150008B8109888E4501D19A420CD88AB3B2FBB3
:10016000F1F001FB102080B258BB122000FB0540CB
:10017000807B012825D1D21A8A42D8BF91B212229F
:1001800002FB0544C9B9D4F80230C9F80430A9F813
:1001900002102DE70A78012ACDD1FF2008701946F8
:1001A00003A80193FFF7F4FB019B06F838301A46C9
:1001B000194603A8FFF7CAFCBDE7D4F8062013448C
:1001C000E3E7122202FB0544D4F80620ADF815300F
:1001D0004FF0FF330492A372E37291E756C0FF1F02
:1001E00013460A46194601F03DBC00BF30B503294D
:1001F000039C04981DD12BB9164A22600422028068
:10020000002030BD40F209418B420FD1022A4FF04D
:1002100000030CD810490C2505FB0313D9681B6992
:1002200051F8221021609B5C0380E9E70123012241
:10023000F0E7072901D9CD2030BD074B03EB810240
:10024000126A2260002AF6D003EB4103B3F8403073
:10025000EAE700BF57C0FF1FA01C010001299FBF94
:10026000034B5B5C1370002088BFCD20704700BF3C
:10027000B0CCFF1F01299DBF024B00205A54CD2056
:10028000704700BFB0CCFF1F19B14B1E58425841F8
:10029000704701207047054B1A788A4204D058787D
:1002A000431A58425841704701207047B0CCFF1F95
:1002B0000020704700487047F01C010001299FBFD3
:1002C000044BC1EBC101C918002094BF1160CD20BF
:1002D000704700BF5BC0FF1F012930B50ED8084D25
:1002E000C1EBC10108231068C45CC818284401335D
:1002F0000F2B00F8084CF6D1002030BDCD2030BDCA
:100300005BC0FF1F01299FBF034B03EB410100208E
:10031000116088BFCD207047B2CCFF1F01299FBF5D
:10032000034B03EB41010020116088BFCD207047D3
:10033000B6CCFF1F01290AD813681878054B03EBC8
:100340004101887013685B78CB7000207047CD2026
:10035000704700BFB0CCFF1F01290AD81368187876
:10036000054B03EB4101887113685B78CB7100206A
:100370007047CD20704700BFB0CCFF1F084B5A78A4
:1003800003F8022BFF210022D1540132072AFBD1AE
:10039000044A0023052199540133072BFBD17047F0
:1003A000BACCFF1FC3CCFF1F00BF7047013AD2B2C7
:1003B000062A10B51C4608D8054B5A70FFF7DEFF19
:1003C0002146BDE81040FFF7C9B9992010BD00BF14
:1003D000BACCFF1F024B00225A70FFF731BA00BFA0
:1003E000BACCFF1F37B50F4C257805B9C1B98DF8C8
:1003F00002308DF800109DF81830ADF803206946E2
:100400009DF81C2000788DF80130FFF737FA9DF831
:1004100000301BB110B92378013B237003B030BD0D
:100420009520FBE7BACCFF1F38B50A4B0D461C7868
:1004300059788C421C4600D14DB929460078FFF707
:10044000D1FA2DB120B923780133237038BD96201D
:1004500038BD00BFBACCFF1F4B1E062B05D8094B79
:1004600019444B78137000207047CB0607D501F074
:100470000F01062903D8034B19444B7AF2E7822077
:10048000704700BFBACCFF1F4B1E062B2DE9F04171
:100490008046174605D8174B19444A700020BDE81E
:1004A000F081CB0622D501F00F05062D1ED8012ABA
:1004B0004FEAD1140F4E06D122462946FFF7C6FA5D
:1004C00035446F72EAE7002AFAD173195B7A012B7F
:1004D000F6D122462946FFF789FB002DF0D184F0A2
:1004E000010229464046FFF781FBE9E78220BDE88B
:1004F000F08100BFBACCFF1F00207047062903D946
:10050000A1F11003072B07D8044B53F82130002B1F
:100510000CBFC42000207047C4207047181D010084
:10052000102810B50C4601D1FFF728FF034B53F8F4
:1005300020300BB120469847002010BD181D010047
:100540001FB5144602228DF807001A8005210DF10F
:100550000F020DF10700FFF77FFF034B9DF80F20FF
:100560001A80236004B010BDCCCCFF1F1FB5144609
:1005700001228DF807001A8004210DF10F020DF100
:100580000700FFF769FF044B9DF80F201A80002039
:10059000236004B010BD00BFCCCCFF1FF0B5002617
:1005A00085B01E8049888DF80700ADF80E10FFF762
:1005B0006BFE18B3BDF80E20114F04ACB2FA82F2F4
:1005C000520901210DF10700FFF75EFF34F8022DFB
:1005D0000421D2B20DF10700FFF756FF7B682246D7
:1005E000012105469DF8070098477B689DF80700A4
:1005F000324602219847284605B0F0BD0425FAE7A7
:10060000CCCCFF1F73B502AC002504F8010D0E46DB
:100610001D80042201212046FFF736FF7288024B1D
:1006200028461A7202B070BDCCCCFF1F13B54C889F
:1006300089888DE80C000B46E2B2210AFFF7D6FD4F
:1006400002B010BD2DE9F04186B017461E4606AA3D
:1006500000238846059303238DF80F0002F8083D18
:1006600001210DF10F00FFF7F7FE98F80050274C1D
:1006700015F0030528D10DF1110206210DF10F002F
:10068000FFF7EAFE9DF811309DF80F0003F0030319
:1006900023800DF11203019305AB00932A462B46EC
:1006A0000221FFF7A3FD059BDB7913F0400F2388A0
:1006B00014BF43F0010323F001032380022333809E
:1006C0003C6006B0BDE8F081012D08D19DF81030E6
:1006D000012B02D198F80430ABB90023EDE7022DCD
:1006E000EED198F8041041F010010DF11202C9B2D8
:1006F0000DF10F00FFF7B0FE9DF8123003F001037B
:1007000023803580DCE7CD20DAE700BFCCCCFF1FAB
:100710007FB500221A800B784E788DF8070013F011
:1007200003030D46C6F3400634D1FEB14B88013BAE
:100730009BB2012B52D80DF10F0206210DF10700DB
:10074000FFF78AFE044670B9AB7801229A409DF803
:100750000F301A43D2B206210DF107008DF80F2099
:10076000FFF792FE0446204604B070BD4E88012E6D
:1007700034D10DF10F0206210DF10700FFF76CFED9
:1007800004460028EFD1AA7896409DF80F2022EA6F
:100790000602E0E7022B21D109798DF80F103246CD
:1007A00041F010010DF10700FFF76EFE6B78002E8F
:1007B00014BF07210821012B044607D19DF80F0023
:1007C000C10900F00F00FFF7ADF90821044B9DF8B7
:1007D00007005B680DF10F029847C4E7CD24C2E71C
:1007E000CCCCFF1F10B500241C800B7803F0030352
:1007F000012B05D18A780979FFF73CFD204610BD11
:10080000042010BD38B515460A7802F00302012A0B
:1008100007D1054C1A8009792246FFF71FFD2C608D
:1008200038BD042038BD00BFCCCCFF1F13B5CD2987
:100830008DF8070007D1012290210DF10700FFF785
:1008400023FE02B010BD0D491C88088A126884423C
:1008500088BF18800C461B889DF807000021FEF712
:100860004DFF94F90A30002BEBDA00231A461946A3
:100870000DF10700FFF76AF9E3E700BFCCCCFF1FDB
:1008800073B5054600266A4601218DF80060019681
:10089000FFF7E2FDAA78434C012A52D16868036849
:1008A000C4F80A304368A07AC4F80E3004F10A0193
:1008B00010F0600F1ED1E27A3B4B53F82240002C1F
:1008C0003DD09DF80000022839D802EB42021344C3
:1008D000034493F83430012B31D10DF1020301AA06
:1008E0002878A0470DF1020301AA01462878FFF7F6
:1008F0009DFF13E0238AADF80230202B17D87BB17F
:1009000002060DD40A68C4F812204A68C4F81620FA
:10091000314604F11A022846FFF718F902B070BDFB
:10092000E46B64B10DF1020301AA2049D8E702A8E3
:100930002B7800F8073D9021FFF7A6FDEEE7CD20CC
:10094000D0E79DF80030042B10D12B78217A02AD2E
:1009500005F8063D2846FFF7D1F901221146284641
:10096000FFF792FD227A03212846E5E794F90A3041
:10097000002BD3DBEB78002BD0D1E66B86B1B5F83A
:10098000093028780833ADF8023004F112010DF176
:10099000020301AAB04701460DF1020301AAA5E72F
:1009A000CD21F9E7CCCCFF1F781D0100D6CCFF1F6D
:1009B000034B5960DA630021024AFFF79DBD00BF77
:1009C000CCCCFF1F8108010007B502AB054A03F834
:1009D000010D002118465160D163FFF78FFD03B070
:1009E0005DF804FBCCCCFF1F00207047354B41F273
:1009F00048015A5822F00D0242F005025A5041F2C5
:100A000004015A5842F480225A5041F234015A5893
:100A100042F480225A5003F52C33602193F894203D
:100A200042F0020283F89420C02283F80021FF22C2
:100A30001A7483F8802083F8882083F884200022A9
:100A400083F88C2083F80C111F491A75080A00F0EE
:100A5000FE0083F8982083F8C02083F8C42083F830
:100A6000C82083F8CC2083F8D02083F8D42083F8E2
:100A7000D82083F8DC2083F8E02083F8E42083F892
:100A8000E82083F8EC2083F8F02083F8F42083F842
:100A9000F82083F8FC2083F89C00C1F30740090E7E
:100AA00083F8B00083F8B41083F8AC201A7783F889
:100AB000082193F8942002F0D40242F0010283F856
:100AC000942070470070044000D6FF1F024B4FF483
:100AD00000729A60704700BF00E100E0034B4FF4E2
:100AE0000072C3F888219A60704700BF00E100E0FF
:100AF00008B5FEF782F910B9FFF7F0FF08BD1B201B
:100B000008BD00BF034B4AF202629A814BF2804259
:100B10009A8170470020054081F0004102E000BF4B
:100B200083F0004330B54FEA41044FEA430594EAAD
:100B3000050F08BF90EA020F1FBF54EA000C55EAE8
:100B4000020C7FEA645C7FEA655C00F0E2804FEAB9
:100B50005454D4EB5555B8BF6D420CDD2C4480EA9B
:100B6000020281EA030382EA000083EA010180EACB
:100B7000020281EA0303362D88BF30BD11F0004F19
:100B80004FEA01314FF4801C4CEA113102D040424F
:100B900061EB410113F0004F4FEA03334CEA13338A
:100BA00002D0524263EB430394EA050F00F0A780A2
:100BB000A4F10104D5F1200E0DDB02FA0EFC22FA9D
:100BC00005F2801841F1000103FA0EF2801843FA91
:100BD00005F359410EE0A5F120050EF1200E012A82
:100BE00003FA0EFC28BF4CF0020C43FA05F3C018C0
:100BF00051EBE37101F0004507D54FF0000EDCF139
:100C0000000C7EEB00006EEB0101B1F5801F1BD3E1
:100C1000B1F5001F0CD349085FEA30004FEA3C0CE5
:100C200004F101044FEA445212F5800F80F09A80DB
:100C3000BCF1004F08BF5FEA500C50F1000041EBDF
:100C4000045141EA050130BD5FEA4C0C404141EBE3
:100C5000010111F4801FA4F10104E9D191F0000F0A
:100C600004BF01460020B1FA81F308BF2033A3F18D
:100C70000B03B3F120020CDA0C3208DD02F1140C84
:100C8000C2F10C0201FA0CF021FA02F10CE002F1BF
:100C90001402D8BFC2F1200C01FA02F120FA0CFCB8
:100CA000DCBF41EA0C019040E41AA2BF01EB045101
:100CB000294330BD6FEA04041F3C1CDA0C340EDCFF
:100CC00004F11404C4F1200220FA04F001FA02F342
:100CD00040EA030021FA04F345EA030130BDC4F100
:100CE0000C04C4F1200220FA02F001FA04F340EAF5
:100CF0000300294630BD21FA04F0294630BD94F0A6
:100D0000000F83F4801306BF81F480110134013D8C
:100D10004EE77FEA645C18BF7FEA655C29D094EAFD
:100D2000050F08BF90EA020F05D054EA000C04BF7B
:100D30001946104630BD91EA030F1EBF0021002066
:100D400030BD5FEA545C05D14000494128BF41F005
:100D5000004130BD14F580043CBF01F5801130BD69
:100D600001F0004545F0FE4141F470014FF00000F4
:100D700030BD7FEA645C1ABF194610467FEA655CA5
:100D80001CBF0B46024650EA013406BF52EA033547
:100D900091EA030F41F4002130BD00BF90F0000F35
:100DA00004BF0021704730B54FF4806404F1320471
:100DB0004FF000054FF0000150E700BF90F0000F2A
:100DC00004BF0021704730B54FF4806404F1320451
:100DD00010F0004548BF40424FF000013EE700BF21
:100DE00042004FEAE2014FEA31014FEA02701FBFB1
:100DF00012F07F4393F07F4F81F06051704792F083
:100E0000000F14BF93F07F4F704730B54FF46074FC
:100E100001F0004521F0004120E700BF50EA010247
:100E200008BF704730B54FF000050AE050EA0102F4
:100E300008BF704730B511F0004502D5404261EB64
:100E400041014FF4806404F132045FEA915C3FF4A5
:100E5000DCAE4FF003025FEADC0C18BF03325FEA3E
:100E6000DC0C18BF033202EBDC02C2F1200300FAF3
:100E700003FC20FA02F001FA03FE40EA0E0021FA18
:100E800002F11444C1E600BF70B54FF0FF0C4CF402
:100E9000E06C1CEA11541DBF1CEA135594EA0C0FB8
:100EA00095EA0C0F00F0DEF82C4481EA030621EAF3
:100EB0004C5123EA4C5350EA013518BF52EA03352E
:100EC00041F4801143F4801338D0A0FB02CE4FF0E0
:100ED0000005E1FB02E506F00042E0FB03E54FF010
:100EE0000006E1FB03569CF0000F18BF4EF0010E08
:100EF000A4F1FF04B6F5007F64F5407404D25FEA04
:100F00004E0E6D4146EB060642EAC62141EA5551B6
:100F10004FEAC52040EA5E504FEACE2EB4F1FD0CF8
:100F200088BFBCF5E06F1ED8BEF1004F08BF5FEA76
:100F3000500E50F1000041EB045170BD06F0004628
:100F400046EA010140EA020081EA0301B4EB5C04D5
:100F5000C2BFD4EB0C0541EA045170BD41F48011CD
:100F60004FF0000E013C00F3AB8014F1360FDEBFF2
:100F7000002001F0004170BDC4F10004203C35DACE
:100F80000C341BDC04F11404C4F1200500FA05F351
:100F900020FA04F001FA05F240EA020001F00042F2
:100FA00021F0004110EBD37021FA04F642EB060168
:100FB0005EEA430E08BF20EAD37070BDC4F10C0492
:100FC000C4F1200500FA04F320FA05F001FA04F256
:100FD00040EA020001F0004110EBD37041F1000142
:100FE0005EEA430E08BF20EAD37070BDC4F120054D
:100FF00000FA05F24EEA020E20FA04F301FA05F2B5
:1010000043EA020321FA04F001F0004121FA04F25C
:1010100020EA020000EBD3705EEA430E08BF20EA2C
:10102000D37070BD94F0000F0FD101F00046400066
:1010300041EB010111F4801F08BF013CF7D041EAE8
:10104000060195F0000F18BF704703F000465200EC
:1010500043EB030313F4801F08BF013DF7D043EABD
:101060000603704794EA0C0F0CEA135518BF95EA73
:101070000C0F0CD050EA410618BF52EA4306D1D1FA
:1010800081EA030101F000414FF0000070BD50EA19
:10109000410606BF1046194652EA430619D094EAA3
:1010A0000C0F02D150EA013613D195EA0C0F05D18D
:1010B00052EA03361CBF104619460AD181EA0301E1
:1010C00001F0004141F0FE4141F470014FF0000099
:1010D00070BD41F0FE4141F4780170BD70B54FF034
:1010E000FF0C4CF4E06C1CEA11541DBF1CEA1355B4
:1010F00094EA0C0F95EA0C0F00F0A7F8A4EB050496
:1011000081EA030E52EA03354FEA013100F088808C
:101110004FEA03334FF0805545EA131343EA126355
:101120004FEA022245EA111545EA10654FEA00260A
:101130000EF000419D4208BF964244F1FD0404F5C3
:10114000407402D25B084FEA3202B61A65EB03051F
:101150005B084FEA32024FF480104FF4002CB6EBDC
:10116000020E75EB030E22BFB61A754640EA0C005C
:101170005B084FEA3202B6EB020E75EB030E22BF9C
:10118000B61A754640EA5C005B084FEA3202B6EBDD
:10119000020E75EB030E22BFB61A754640EA9C009C
:1011A0005B084FEA3202B6EB020E75EB030E22BF6C
:1011B000B61A754640EADC0055EA060E18D04FEA2A
:1011C000051545EA16754FEA06164FEAC30343EACA
:1011D00052734FEAC2025FEA1C1CC0D111F4801F97
:1011E0000BD141EA00014FF000004FF0004CB6E790
:1011F00011F4801F04BF01430020B4F1FD0C88BF2F
:10120000BCF5E06F3FF6AFAEB5EB030C04BFB6EB39
:10121000020C5FEA500C50F1000041EB045170BD2C
:101220000EF0004E4EEA113114EB5C04C2BFD4EB59
:101230000C0541EA045170BD41F480114FF0000EDD
:10124000013C90E645EA060E8DE60CEA135594EA59
:101250000C0F08BF95EA0C0F3FF43BAF94EA0C0F5C
:101260000AD150EA01347FF434AF95EA0C0F7FF4D1
:1012700025AF104619462CE795EA0C0F06D152EA25
:1012800003353FF4FDAE1046194622E750EA410609
:1012900018BF52EA43067FF4C5AE50EA41047FF41A
:1012A0000DAF52EA43057FF4EBAE12E74FEA41027D
:1012B00012F5001215D211D56FF47873B3EB6252A8
:1012C00012D94FEAC12343F0004343EA505311F0CF
:1012D000004F23FA02F018BF404270474FF0000061
:1012E000704750EA013005D111F0004008BF6FF09F
:1012F000004070474FF00000704700BF4FEA4102C6
:10130000B2F1E04324BFB3F5001CDCF1FE5C0DD963
:1013100001F0004C4FEAC0024CEA5070B2F1004FAD
:1013200040EB830008BF20F00100704711F0804FB0
:1013300021D113F13872BCBF01F00040704741F475
:1013400080114FEA5252C2F11802C2F1200C10FA79
:101350000CF320FA02F018BF40F001004FEAC1235D
:101360004FEAD32303FA0CFC40EA0C0023FA02F301
:101370004FEA4303CCE77FEA625307D150EA0133D7
:101380001EBF4FF0FE4040F44000704701F00040A7
:1013900040F0FE4040F40000704700BF80F0004085
:1013A00002E000BF81F0004142001FBF5FEA41033D
:1013B00092EA030F7FEA226C7FEA236C6AD04FEA3D
:1013C0001262D2EB1363C1BFD21841404840414082
:1013D000B8BF5B42192B88BF704710F0004F40F434
:1013E000000020F07F4018BF404211F0004F41F450
:1013F000000121F07F4118BF494292EA030F3FD01C
:10140000A2F1010241FA03FC10EB0C00C3F120032E
:1014100001FA03F100F0004302D5494260EB4000BD
:10142000B0F5000F13D3B0F1807F06D340084FEA28
:10143000310102F10102FE2A51D2B1F1004F40EB1D
:10144000C25008BF20F0010040EA03007047490085
:1014500040EB000010F4000FA2F10102EDD1B0FA50
:1014600080FCACF1080CB2EB0C0200FA0CF0AABF45
:1014700000EBC25052421843BCBFD04018437047E3
:1014800092F0000F81F4000106BF80F400000132E9
:10149000013BB5E74FEA41037FEA226C18BF7FEAC0
:1014A000236C21D092EA030F04D092F0000F08BF02
:1014B0000846704790EA010F1CBF0020704712F0E9
:1014C0007F4F04D1400028BF40F00040704712F128
:1014D00000723CBF00F50000704700F0004343F08D
:1014E000FE4040F4000070477FEA226216BF0846C3
:1014F0007FEA23630146420206BF5FEA412390EA86
:10150000010F40F4800070474FF0000304E000BF7B
:1015100010F0004348BF40425FEA000C08BF70472C
:1015200043F0964301464FF000001CE050EA0102F0
:1015300008BF70474FF000030AE000BF50EA010205
:1015400008BF704711F0004302D5404261EB4101F2
:101550005FEA010C02BF84460146002043F0B64317
:1015600008BFA3F18053A3F50003BCFA8CF2083A3C
:10157000A3EBC25310DB01FA02FC634400FA02FC45
:10158000C2F12002BCF1004F20FA02F243EB02004C
:1015900008BF20F00100704702F1200201FA02FCAE
:1015A000C2F1200250EA4C0021FA02F243EB0200A1
:1015B00008BF20EADC7070474FF0FF0C1CEAD052E5
:1015C0001EBF1CEAD15392EA0C0F93EA0C0F6FD0A6
:1015D0001A4480EA010C400218BF5FEA41211ED084
:1015E0004FF0006343EA501043EA5111A0FB013170
:1015F0000CF00040B1F5000F3EBF490041EAD37145
:101600005B0040EA010062F17F02FD2A1DD8B3F1C0
:10161000004F40EBC25008BF20F00100704790F02F
:10162000000F0CF0004C08BF49024CEA502040EA81
:1016300051207F3AC2BFD2F1FF0340EAC250704747
:1016400040F400004FF00003013A5DDC12F1190F85
:10165000DCBF00F000407047C2F10002410021FAF7
:1016600002F1C2F1200200FA02FC5FEA310040F10F
:10167000000053EA4C0308BF20EADC70704792F088
:10168000000F00F0004C02BF400010F4000F013AC0
:10169000F9D040EA0C0093F0000F01F0004C02BFBB
:1016A000490011F4000F013BF9D041EA0C018FE72A
:1016B0000CEAD15392EA0C0F18BF93EA0C0F0AD030
:1016C00030F0004C18BF31F0004CD8D180EA010056
:1016D00000F00040704790F0000F17BF90F0004FEF
:1016E000084691F0000F91F0004F14D092EA0C0FD1
:1016F00001D142020FD193EA0C0F03D14B0218BF64
:10170000084608D180EA010000F0004040F0FE40A9
:1017100040F40000704740F0FE4040F44000704745
:101720004FF0FF0C1CEAD0521EBF1CEAD15392EAC4
:101730000C0F93EA0C0F69D0A2EB030280EA010CB4
:1017400049024FEA402037D04FF0805343EA11114D
:1017500043EA10130CF000408B4238BF5B0042F1AB
:101760007D024FF4000C8B4224BF5B1A40EA0C0050
:10177000B3EB510F24BFA3EB510340EA5C00B3EB82
:10178000910F24BFA3EB910340EA9C00B3EBD10F70
:1017900024BFA3EBD10340EADC001B0118BF5FEAC2
:1017A0001C1CE0D1FD2A3FF650AF8B4240EBC250EB
:1017B00008BF20F0010070470CF0004C4CEA5020AC
:1017C0007F32C2BFD2F1FF0340EAC250704740F4FB
:1017D00000004FF00003013A37E792F0000F00F0ED
:1017E000004C02BF400010F4000F013AF9D040EA6B
:1017F0000C0093F0000F01F0004C02BF490011F4FF
:10180000000F013BF9D041EA0C0195E70CEAD153F6
:1018100092EA0C0F08D142027FF47DAF93EA0C0FDD
:101820007FF470AF084676E793EA0C0F04D14B02C1
:101830003FF44CAF08466EE730F0004C18BF31F073
:10184000004CCAD130F000427FF45CAF31F000436D
:101850007FF43CAF5FE700BF4FF0FF3C06E000BF06
:101860004FF0010C02E000BF4FF0010C4DF804CD29
:101870004FEA40024FEA41037FEA226C18BF7FEA39
:10188000236C11D001B052EA530C18BF90EA010F3B
:1018900058BFB2EB030088BFC81738BF6FEAE170CA
:1018A00018BF40F0010070477FEA226C02D15FEA66
:1018B000402C05D17FEA236CE4D15FEA412CE1D0D2
:1018C0005DF8040B704700BF844608466146FFE799
:1018D0000FB5FFF7C9FF002848BF10F1000F0FBD7B
:1018E0004DF808EDFFF7F4FF0CBF012000205DF874
:1018F00008FB00BF4DF808EDFFF7EAFF34BF0120F9
:1019000000205DF808FB00BF4DF808EDFFF7E0FF91
:1019100094BF012000205DF808FB00BF4DF808EDE2
:10192000FFF7D2FF94BF012000205DF808FB00BF45
:101930004DF808EDFFF7C8FF34BF012000205DF827
:1019400008FB00BF42000ED2B2F1FE4F0BD34FF0A6
:101950009E03B3EB126209D44FEA002343F0004325
:1019600023FA02F070474FF00000704712F1610F48
:1019700001D1420202D14FF0FF3070474FF000001A
:10198000704700BFFDF707F9002103E00A4B5B58E1
:101990004350043109480A4B42189A42F6D3094A87
:1019A00002E0002313600432074B9A42F9D300F09F
:1019B0000DF8804770470000041E010008C0FF1F9B
:1019C0006CC5FF1F00C6FF1F24DAFF1F224C08B59D
:1019D000F6F757FDF6F7BEFDF6F772FFF6F789FF4B
:1019E000F6F784FEF7F73CFAFCF754FEF7F7BBFC7A
:1019F000F7F720F8E08CF7F71EF92078F6F790FE5D
:101A0000E078F6F7FDFEF7F707FA21896079228A78
:101A1000FCF794FEF8F7F8F8F8F7DCFAFDF75AF857
:101A20000E4B04229A60FBF771FBFCF707F80C4B96
:101A300020229A60FBF766FCFCF71EF8FBF7FFFF1D
:101A4000F7F7A6F9F7F7D8F90028F3D0F8F7C2FAB4
:101A5000FBF75CFBEEE700BF0CC0FF1FC0F00F40C0
:101A600000F10F4070B4860746D0541E002A41D0C2
:101A7000CAB2034602E014F1FF343BD303F8012B52
:101A80009D07F8D1032C2ED9CDB245EA05250F2CA0
:101A900045EA054519D903F110022646103E0F2EDE
:101AA00042F8105C42F80C5C42F8085C42F8045CB6
:101AB00002F11002F2D8A4F1100222F00F0204F099
:101AC0000F041032032C13440DD91E462246043A4B
:101AD000032A46F8045BFAD8221F22F003020432DC
:101AE000134404F003042CB1C9B21C4403F8011BD5
:101AF0009C42FBD170BC704714460346C2E700BF4E
:101B0000024B13B1024800F005B870470000000016
:101B1000211B0100002301461A46184600F01EB89A
:101B200038B50A4C0A4D641BA4100AD004F1804356
:101B3000013B05EB8305013C55F804399847002C1F
:101B4000F9D1BDE8384000F051B900BF041E0100D2
:101B5000001E0100704700BF704700BF2DE9F84329
:101B60002C4D0646286898460F469146FFF7F2FF2F
:101B7000294B1C68D4F84831002B3ED05A681F2AE4
:101B80001CDC02F1010E76B103EB82010124C1F8E5
:101B90008890D3F8880194402043022EC3F888012E
:101BA000C1F8088123D00232C3F804E0286843F862
:101BB0002270FFF7D1FF0020BDE8F883174B0BB36D
:101BC0004FF4C870AFF300800346D8B1D4F8482171
:101BD0000260002141600A46C4F848014FF0010E3E
:101BE000C0F88811C0F88C11002EDCD0CCE7D3F8F7
:101BF0008C110C43C3F88C41D5E704F5A673C4F8E7
:101C00004831BBE72868FFF7A7FF4FF0FF30BDE87A
:101C1000F88300BF68C5FF1FDC1D01000000000045
:101C20008025000040380000004B0000807000005C
:101C30000096000000E10000002C010000C201003D
:101C40000084030090D0030020A1070040420F0051
:101C5000F40100006400000001800808000000009A
:101C6000006400000000000000000000C800000048
:101C70000000000000000000010003E80000000078
:101C800000000003E800000000000200FA06000364
:101C90000000000000370600000000000000000007
:101CA00057C0FF1F0400000009040000041D0100CC
:101CB000141D0100000000000000000000000000F2
:101CC000000000002EC1FF1FEBC0FF1F000000003E
:101CD0000000000000000000000000000000000004
:101CE000000012004300000000000000000000009F
:101CF00003010201100002020010000303011000A2
:101D00000001000057C0FF1FB1C0FF1F8BC0FF1FA5
:101D100069C0FF1F043A2622810801007DF10000FE
:101D200015F2000085EF0000A9030100A9030100DE
:101D3000A9030100A9030100A9030100A9030100EF
:101D4000A9030100A9030100A9030100A9030100DF
:101D5000A9030100A903010007F500009DF400009C
:101D6000FDF40000C9F400009DF40000A903010087
:101D700089F4000075F50000450601001107010017
:101D8000000000001107010000000000050601002E
:101D90002D060100000000006D0501009D050100F9
:101DA00005080100E50701004105010001010001EE
:101DB000010000000001010000000000010101011C
:101DC000010000000101000101000100000100000C
:101DD00001000031313130563130380040C1FF1F31
:101DE000F8B500BFF8BC08BC9E467047F8B500BF08
:081DF000F8BC08BC9E467047D8
:081DF800011B0100358400000D
:041E00001184000049
:101E0400D31D0100000102000008000001000000D1
:101E140002000000000000000000000000000000BC
:101E240000000000000000000000070000000000A7
:101E3400000000000000000000000000000000009E
:101E440000000000A1200000000002000000FF04C8
:101E540003090400C20100000008000000000000A3
:101E64000022034200410044002000530054005269
:101E74000049004E004700200049004E0044004540
:101E8400005800260353007400650070007000655C
:101E940000720020004D006F0074006F007200207B
:101EA4000044006500760020003A035400520049C3
:101EB400004E0041004D004900430020004D006FDA
:101EC40000740069006F006E00200043006F006E14
:101ED40000740072006F006C0020002000200020BD
:101EE40000200009024300020100C032090400007E
:101EF400010202000005240010010524010101046F
:101F040024020605240600010705830310000A09BC
:101F1400040100020A000000070581021000000706
:101F240005020210000012010002020000103C2A07
:101F34000001020001020001000000002CC4FF1F88
:101F440094C4FF1FFCC4FF1F000000000000000039
:101F5400000000000000000000000000000000007D
:101F6400000000000000000000000000000000006D
:101F7400000000000000000000000000000000005D
:101F8400000000000000000000000000000000004D
:101F9400000000000000000000000000000000003D
:101FA400000000000000000000000000000000002D
:101FB400000000000000000000000000000000001D
:101FC400000000000000000000000000000000000D
:101FD40000000000000000000000000000000000FD
:101FE40001000000000000000E33CDAB34126DE69A
:101FF400ECDE05000B000000000000000000000003
:1020040000000000000000000000000000000000CC
:1020140000000000000000000000000000000000BC
:1020240000000000000000000000000000000000AC
:10203400000000000000000000000000000000009C
:0423640000DAFF1F7D
:10236800041E010008C0FF1F6405000000000000F3
:0823780000000000000000005D
:020000020000FC
:020000041FFFDC
:04C00000000000003C
:04000003100019854B
:00000001FF
